 net

 Timestamp is 7219a72c (reproducible build file hash)

 Preferred load address is 0000000180000000

 Start         Length     Name                   Class
 0001:00000000 00006b40H .text$mn                CODE
 0001:00006b40 00000036H .text$mn$00             CODE
 0001:00006b76 00000092H .text$x                 CODE
 0002:00000000 00000390H .idata$5                DATA
 0002:00000390 00000038H .00cfg                  DATA
 0002:000003c8 00000008H .CRT$XCA                DATA
 0002:000003d0 00000008H .CRT$XCZ                DATA
 0002:000003d8 00000008H .CRT$XIA                DATA
 0002:000003e0 00000008H .CRT$XIZ                DATA
 0002:000003e8 00000008H .CRT$XPA                DATA
 0002:000003f0 00000008H .CRT$XPZ                DATA
 0002:000003f8 00000008H .CRT$XTA                DATA
 0002:00000400 00000010H .CRT$XTZ                DATA
 0002:00000408 00000000H .gehcont$y              DATA
 0002:00000408 00000000H .gfids$y                DATA
 0002:00000410 000016f0H .rdata                  DATA
 0002:00001b00 00000000H .rdata$CastGuardVftablesA DATA
 0002:00001b00 00000000H .rdata$CastGuardVftablesC DATA
 0002:00001b00 00000094H .rdata$voltmd           DATA
 0002:00001b94 0000032cH .rdata$zzzdbg           DATA
 0002:00001ec0 00000008H .rtc$IAA                DATA
 0002:00001ec8 00000008H .rtc$IZZ                DATA
 0002:00001ed0 00000008H .rtc$TAA                DATA
 0002:00001ed8 00000008H .rtc$TZZ                DATA
 0002:00001ee0 000005a4H .xdata                  DATA
 0002:00002484 00000040H .didat$2                DATA
 0002:000024c4 00000024H .didat$3                DATA
 0002:000024e8 000000b8H .didat$4                DATA
 0002:000025a0 000001d0H .didat$6                DATA
 0002:00002770 000000c0H .didat$7                DATA
 0002:00002830 00000a4cH .edata                  DATA
 0002:0000327c 000000dcH .idata$2                DATA
 0002:00003358 00000018H .idata$3                DATA
 0002:00003370 00000390H .idata$4                DATA
 0002:00003700 0000076cH .idata$6                DATA
 0003:00000000 000000e0H .data                   DATA
 0003:000000e0 000000c0H .didat$5                DATA
 0003:000001a0 000007b0H .bss                    DATA
 0004:00000000 000005d0H .pdata                  DATA
 0005:00000000 00000060H .rsrc$01                DATA
 0005:00000060 00000318H .rsrc$02                DATA

  Address         Publics by Value              Rva+Base               Lib:Object

 0000:00000000       __AbsoluteZero             0000000000000000     <absolute>
 0000:00000000       ___safe_se_handler_count   0000000000000000     <absolute>
 0000:00000000       ___safe_se_handler_table   0000000000000000     <absolute>
 0000:00000000       __arm64x_extra_rfe_table   0000000000000000     <absolute>
 0000:00000000       __arm64x_extra_rfe_table_size 0000000000000000     <absolute>
 0000:00000000       __arm64x_native_entrypoint 0000000000000000     <absolute>
 0000:00000000       __arm64x_redirection_metadata 0000000000000000     <absolute>
 0000:00000000       __arm64x_redirection_metadata_count 0000000000000000     <absolute>
 0000:00000000       __dynamic_value_reloc_table 0000000000000000     <absolute>
 0000:00000000       __enclave_config           0000000000000000     <absolute>
 0000:00000000       __guard_check_icall_a64n_fptr 0000000000000000     <absolute>
 0000:00000000       __guard_eh_cont_count      0000000000000000     <absolute>
 0000:00000000       __guard_eh_cont_table      0000000000000000     <absolute>
 0000:00000000       __guard_fids_count         0000000000000000     <absolute>
 0000:00000000       __guard_fids_table         0000000000000000     <absolute>
 0000:00000000       __guard_iat_count          0000000000000000     <absolute>
 0000:00000000       __guard_iat_table          0000000000000000     <absolute>
 0000:00000000       __guard_longjmp_count      0000000000000000     <absolute>
 0000:00000000       __guard_longjmp_table      0000000000000000     <absolute>
 0000:00000000       __hybrid_auxiliary_delayload_iat 0000000000000000     <absolute>
 0000:00000000       __hybrid_auxiliary_delayload_iat_copy 0000000000000000     <absolute>
 0000:00000000       __hybrid_auxiliary_iat     0000000000000000     <absolute>
 0000:00000000       __hybrid_auxiliary_iat_copy 0000000000000000     <absolute>
 0000:00000000       __hybrid_code_map          0000000000000000     <absolute>
 0000:00000000       __hybrid_code_map_count    0000000000000000     <absolute>
 0000:00000000       __hybrid_image_info_bitfield 0000000000000000     <absolute>
 0000:00000000       __x64_code_ranges_to_entry_points 0000000000000000     <absolute>
 0000:00000000       __x64_code_ranges_to_entry_points_count 0000000000000000     <absolute>
 0000:00000100       __guard_flags              0000000000000100     <absolute>
 0000:00000000       __ImageBase                0000000180000000     <linker-defined>
 0001:00000000       Java_sun_net_spi_DefaultProxySelector_getSystemProxies 0000000180001000 f   DefaultProxySelector.obj
 0001:0000054c       Java_sun_net_spi_DefaultProxySelector_init 000000018000154c f   DefaultProxySelector.obj
 0001:00000590       __local_stdio_printf_options 0000000180001590 f i DefaultProxySelector.obj
 0001:00000598       __local_stdio_scanf_options 0000000180001598 f i DefaultProxySelector.obj
 0001:000006ec       swprintf                   00000001800016ec f i DefaultProxySelector.obj
 0001:00000740       swscanf                    0000000180001740 f i DefaultProxySelector.obj
 0001:0000078c       Java_java_net_Inet4Address_init 000000018000178c f   Inet4Address.obj
 0001:00000808       Java_java_net_Inet4AddressImpl_getHostByAddr 0000000180001808 f   Inet4AddressImpl.obj
 0001:0000091c       Java_java_net_Inet4AddressImpl_getLocalHostName 000000018000191c f   Inet4AddressImpl.obj
 0001:0000091c       Java_java_net_Inet6AddressImpl_getLocalHostName 000000018000191c f   Inet6AddressImpl.obj
 0001:00000988       Java_java_net_Inet4AddressImpl_isReachable0 0000000180001988 f   Inet4AddressImpl.obj
 0001:00000b38       Java_java_net_Inet4AddressImpl_lookupAllHostAddr 0000000180001b38 f   Inet4AddressImpl.obj
 0001:00001224       Java_java_net_Inet6Address_init 0000000180002224 f   Inet6Address.obj
 0001:000013b0       Java_java_net_Inet6AddressImpl_getHostByAddr 00000001800023b0 f   Inet6AddressImpl.obj
 0001:00001510       Java_java_net_Inet6AddressImpl_isReachable0 0000000180002510 f   Inet6AddressImpl.obj
 0001:000016dc       Java_java_net_Inet6AddressImpl_lookupAllHostAddr 00000001800026dc f   Inet6AddressImpl.obj
 0001:00001e20       Java_java_net_InetAddress_init 0000000180002e20 f   InetAddress.obj
 0001:00001fa0       Java_java_net_InetAddress_isIPv4Available 0000000180002fa0 f   InetAddress.obj
 0001:00001fa8       Java_java_net_InetAddress_isIPv6Supported 0000000180002fa8 f   InetAddress.obj
 0001:00001fb0       Java_sun_net_www_protocol_http_ntlm_NTLMAuthSequence_getCredentialsHandle 0000000180002fb0 f   NTLMAuthSequence.obj
 0001:00002178       Java_sun_net_www_protocol_http_ntlm_NTLMAuthSequence_getNextToken 0000000180003178 f   NTLMAuthSequence.obj
 0001:000023e4       Java_sun_net_www_protocol_http_ntlm_NTLMAuthSequence_initFirst 00000001800033e4 f   NTLMAuthSequence.obj
 0001:000024f8       Java_sun_net_www_protocol_http_ntlm_NTLMAuthentication_isTrustedSite0 00000001800034f8 f   NTLMAuthentication.obj
 0001:00002630       Java_sun_net_www_protocol_http_ntlm_NTLMAuthentication_isTrustedSiteAvailable 0000000180003630 f   NTLMAuthentication.obj
 0001:00002668       Java_java_net_NetworkInterface_boundInetAddress0 0000000180003668 f   NetworkInterface.obj
 0001:00002744       Java_java_net_NetworkInterface_getAll 0000000180003744 f   NetworkInterface.obj
 0001:00002870       Java_java_net_NetworkInterface_getByIndex0 0000000180003870 f   NetworkInterface.obj
 0001:000028e4       Java_java_net_NetworkInterface_getByInetAddress0 00000001800038e4 f   NetworkInterface.obj
 0001:00002a34       Java_java_net_NetworkInterface_getByName0 0000000180003a34 f   NetworkInterface.obj
 0001:00002b00       Java_java_net_NetworkInterface_getMTU0 0000000180003b00 f   NetworkInterface.obj
 0001:00002b98       Java_java_net_NetworkInterface_getMacAddr0 0000000180003b98 f   NetworkInterface.obj
 0001:00002c74       Java_java_net_NetworkInterface_init 0000000180003c74 f   NetworkInterface.obj
 0001:00002eec       Java_java_net_NetworkInterface_isLoopback0 0000000180003eec f   NetworkInterface.obj
 0001:00002f84       Java_java_net_NetworkInterface_isP2P0 0000000180003f84 f   NetworkInterface.obj
 0001:0000301c       Java_java_net_NetworkInterface_isUp0 000000018000401c f   NetworkInterface.obj
 0001:000030c0       Java_java_net_NetworkInterface_supportsMulticast0 00000001800040c0 f   NetworkInterface.obj
 0001:000030c0       __acrt_initialize          00000001800040c0 f   MSVCRT:ucrt_stubs.obj
 0001:000030c0       __acrt_thread_attach       00000001800040c0 f   MSVCRT:ucrt_stubs.obj
 0001:000030c0       __acrt_thread_detach       00000001800040c0 f   MSVCRT:ucrt_stubs.obj
 0001:000030c0       __acrt_uninitialize        00000001800040c0 f   MSVCRT:ucrt_stubs.obj
 0001:000030c0       __acrt_uninitialize_critical 00000001800040c0 f   MSVCRT:ucrt_stubs.obj
 0001:000030c0       __scrt_stub_for_acrt_initialize 00000001800040c0 f   MSVCRT:ucrt_stubs.obj
 0001:000030c0       __scrt_stub_for_acrt_thread_attach 00000001800040c0 f   MSVCRT:ucrt_stubs.obj
 0001:000030c0       __scrt_stub_for_acrt_thread_detach 00000001800040c0 f   MSVCRT:ucrt_stubs.obj
 0001:000030c0       __scrt_stub_for_acrt_uninitialize 00000001800040c0 f   MSVCRT:ucrt_stubs.obj
 0001:000030c0       __scrt_stub_for_acrt_uninitialize_critical 00000001800040c0 f   MSVCRT:ucrt_stubs.obj
 0001:000030c0       __vcrt_initialize          00000001800040c0 f   MSVCRT:ucrt_stubs.obj
 0001:000030c0       __vcrt_thread_attach       00000001800040c0 f   MSVCRT:ucrt_stubs.obj
 0001:000030c0       __vcrt_thread_detach       00000001800040c0 f   MSVCRT:ucrt_stubs.obj
 0001:000030c0       __vcrt_uninitialize        00000001800040c0 f   MSVCRT:ucrt_stubs.obj
 0001:000030c0       __vcrt_uninitialize_critical 00000001800040c0 f   MSVCRT:ucrt_stubs.obj
 0001:000039b0       Java_sun_net_dns_ResolverConfigurationImpl_init0 00000001800049b0 f   ResolverConfigurationImpl.obj
 0001:00003a14       Java_sun_net_dns_ResolverConfigurationImpl_loadDNSconfig0 0000000180004a14 f   ResolverConfigurationImpl.obj
 0001:00003ae4       Java_sun_net_dns_ResolverConfigurationImpl_notifyAddrChange0 0000000180004ae4 f   ResolverConfigurationImpl.obj
 0001:00003e0c       strappend                  0000000180004e0c f   ResolverConfigurationImpl.obj
 0001:00003e8c       JNI_OnLoad                 0000000180004e8c f   net_util.obj
 0001:00003f78       NET_GetPortFromSockaddr    0000000180004f78 f   net_util.obj
 0001:00003f98       NET_SockaddrEqualsInetAddress 0000000180004f98 f   net_util.obj
 0001:000040b0       NET_SockaddrToInetAddress  00000001800050b0 f   net_util.obj
 0001:0000425c       addressesInSystemOrder     000000018000525c f   net_util.obj
 0001:00004268       getInet6Address_ipaddress  0000000180005268 f   net_util.obj
 0001:00004314       getInet6Address_scopeid    0000000180005314 f   net_util.obj
 0001:00004378       getInetAddress_addr        0000000180005378 f   net_util.obj
 0001:000043f0       getInetAddress_family      00000001800053f0 f   net_util.obj
 0001:00004468       initInetAddressIDs         0000000180005468 f   net_util.obj
 0001:000044d8       ipv4_available             00000001800054d8 f   net_util.obj
 0001:000044e0       ipv6_available             00000001800054e0 f   net_util.obj
 0001:000044e8       lookupCharacteristicsToAddressFamily 00000001800054e8 f   net_util.obj
 0001:00004508       reuseport_available        0000000180005508 f   net_util.obj
 0001:00004510       setInet6Address_ipaddress  0000000180005510 f   net_util.obj
 0001:000045ec       setInet6Address_scopeid    00000001800055ec f   net_util.obj
 0001:00004674       setInet6Address_scopeifname 0000000180005674 f   net_util.obj
 0001:000046dc       setInetAddress_addr        00000001800056dc f   net_util.obj
 0001:00004750       setInetAddress_family      0000000180005750 f   net_util.obj
 0001:000047c4       setInetAddress_hostName    00000001800057c4 f   net_util.obj
 0001:00004850       DllMain                    0000000180005850 f   net_util_md.obj
 0001:000048b0       IPv4_supported             00000001800058b0 f   net_util_md.obj
 0001:000048e4       IPv6_supported             00000001800058e4 f   net_util_md.obj
 0001:00004918       IsWindows10RS3OrGreater    0000000180005918 f   net_util_md.obj
 0001:000049d4       NET_Bind                   00000001800059d4 f   net_util_md.obj
 0001:00004a08       NET_EnableFastTcpLoopback  0000000180005a08 f   net_util_md.obj
 0001:00004a64       NET_EnableFastTcpLoopbackConnect 0000000180005a64 f   net_util_md.obj
 0001:00004af0       NET_GetSockOpt             0000000180005af0 f   net_util_md.obj
 0001:00004b78       NET_IPv4MappedToIPv4       0000000180005b78 f   net_util_md.obj
 0001:00004b98       NET_InetAddressToSockaddr  0000000180005b98 f   net_util_md.obj
 0001:00004d5c       NET_IsEqual                0000000180005d5c f   net_util_md.obj
 0001:00004d88       NET_IsIPv4Mapped           0000000180005d88 f   net_util_md.obj
 0001:00004da8       NET_MapSocketOption        0000000180005da8 f   net_util_md.obj
 0001:00004dec       NET_MapSocketOptionV6      0000000180005dec f   net_util_md.obj
 0001:00004e20       NET_SetSockOpt             0000000180005e20 f   net_util_md.obj
 0001:00004f00       NET_Socket                 0000000180005f00 f   net_util_md.obj
 0001:00004f30       NET_SocketAvailable        0000000180005f30 f   net_util_md.obj
 0001:00004f64       NET_ThrowByNameWithLastError 0000000180005f64 f   net_util_md.obj
 0001:00004f6c       NET_ThrowNew               0000000180005f6c f   net_util_md.obj
 0001:00005080       NET_Wait                   0000000180006080 f   net_util_md.obj
 0001:00005224       NET_WinBind                0000000180006224 f   net_util_md.obj
 0001:00005264       __scrt_stub_for_is_c_termination_complete 0000000180006264 f   MSVCRT:ucrt_stubs.obj
 0001:00005264       _is_c_termination_complete 0000000180006264 f   MSVCRT:ucrt_stubs.obj
 0001:00005264       reuseport_supported        0000000180006264 f   net_util_md.obj
 0001:00005268       setExclusiveBind           0000000180006268 f   net_util_md.obj
 0001:000052d0       snprintf                   00000001800062d0 f i net_util_md.obj
 0001:00005328       initJavaClass              0000000180006328 f   proxy_util.obj
 0001:000054cc       jio_snprintf               00000001800064cc f   jvm:jvm.dll
 0001:000054d2       JVM_CurrentTimeMillis      00000001800064d2 f   jvm:jvm.dll
 0001:000054d8       __imp_load_AcquireCredentialsHandleA 00000001800064d8 f   secur32:Secur32.dll
 0001:000054e4       AcquireCredentialsHandleA  00000001800064e4 f   secur32:Secur32.dll
 0001:000054ea       __tailMerge_secur32_dll    00000001800064ea     secur32:Secur32.dll
 0001:00005563       __imp_load_FreeCredentialsHandle 0000000180006563 f   secur32:Secur32.dll
 0001:0000556f       __imp_load_InitializeSecurityContextA 000000018000656f f   secur32:Secur32.dll
 0001:0000557b       InitializeSecurityContextA 000000018000657b f   secur32:Secur32.dll
 0001:00005581       __imp_load_CompleteAuthToken 0000000180006581 f   secur32:Secur32.dll
 0001:0000558d       CompleteAuthToken          000000018000658d f   secur32:Secur32.dll
 0001:00005593       __imp_load_DeleteSecurityContext 0000000180006593 f   secur32:Secur32.dll
 0001:0000559f       __imp_load_IcmpCreateFile  000000018000659f f   iphlpapi:IPHLPAPI.DLL
 0001:000055ab       __tailMerge_iphlpapi_dll   00000001800065ab     iphlpapi:IPHLPAPI.DLL
 0001:00005624       __imp_load_IcmpCloseHandle 0000000180006624 f   iphlpapi:IPHLPAPI.DLL
 0001:00005630       __imp_load_IcmpSendEcho    0000000180006630 f   iphlpapi:IPHLPAPI.DLL
 0001:0000563c       __imp_load_IcmpSendEcho2Ex 000000018000663c f   iphlpapi:IPHLPAPI.DLL
 0001:00005648       __imp_load_Icmp6CreateFile 0000000180006648 f   iphlpapi:IPHLPAPI.DLL
 0001:00005654       __imp_load_Icmp6SendEcho2  0000000180006654 f   iphlpapi:IPHLPAPI.DLL
 0001:00005660       __imp_load_GetIfEntry2     0000000180006660 f   iphlpapi:IPHLPAPI.DLL
 0001:0000566c       __imp_load_GetIfTable2     000000018000666c f   iphlpapi:IPHLPAPI.DLL
 0001:00005678       __imp_load_GetUnicastIpAddressTable 0000000180006678 f   iphlpapi:IPHLPAPI.DLL
 0001:00005684       __imp_load_GetAnycastIpAddressTable 0000000180006684 f   iphlpapi:IPHLPAPI.DLL
 0001:00005690       __imp_load_FreeMibTable    0000000180006690 f   iphlpapi:IPHLPAPI.DLL
 0001:0000569c       __imp_load_ConvertInterfaceNameToLuidW 000000018000669c f   iphlpapi:IPHLPAPI.DLL
 0001:000056a8       __imp_load_ConvertInterfaceLuidToNameW 00000001800066a8 f   iphlpapi:IPHLPAPI.DLL
 0001:000056b4       __imp_load_ConvertLengthToIpv4Mask 00000001800066b4 f   iphlpapi:IPHLPAPI.DLL
 0001:000056c0       __imp_load_NotifyAddrChange 00000001800066c0 f   iphlpapi:IPHLPAPI.DLL
 0001:000056cc       __imp_load_GetAdaptersAddresses 00000001800066cc f   iphlpapi:IPHLPAPI.DLL
 0001:000056d8       ?DloadAcquireSectionWriteAccess@@YAXXZ 00000001800066d8 f i delayimp:delayhlp.obj
 0001:00005784       ?DloadGetSRWLockFunctionPointers@@YAEXZ 0000000180006784 f i delayimp:delayhlp.obj
 0001:00005824       ?DloadMakePermanentImageCommit@@YAXPEAX_K@Z 0000000180006824 f i delayimp:delayhlp.obj
 0001:000058bc       ?DloadObtainSection@@YAPEAXPEAK0@Z 00000001800068bc f i delayimp:delayhlp.obj
 0001:00005958       ?DloadProtectSection@@YAXKPEAK@Z 0000000180006958 f i delayimp:delayhlp.obj
 0001:000059e8       ?DloadReleaseSectionWriteAccess@@YAXXZ 00000001800069e8 f i delayimp:delayhlp.obj
 0001:00005a7c       __delayLoadHelper2         0000000180006a7c f   delayimp:delayhlp.obj
 0001:00005d52       JNU_ThrowOutOfMemoryError  0000000180006d52 f   java:java.dll
 0001:00005d58       JNU_ThrowByName            0000000180006d58 f   java:java.dll
 0001:00005d5e       JNU_ThrowNullPointerException 0000000180006d5e f   java:java.dll
 0001:00005d64       JNU_NewStringPlatform      0000000180006d64 f   java:java.dll
 0001:00005d6a       JNU_GetStringPlatformCharsStrict 0000000180006d6a f   java:java.dll
 0001:00005d70       JNU_ReleaseStringPlatformChars 0000000180006d70 f   java:java.dll
 0001:00005d76       JDK_LoadSystemLibrary      0000000180006d76 f   java:java.dll
 0001:00005d7c       JNU_ThrowInternalError     0000000180006d7c f   java:java.dll
 0001:00005d82       JNU_ThrowByNameWithMessageAndLastError 0000000180006d82 f   java:java.dll
 0001:00005d88       __GSHandlerCheck           0000000180006d88 f   MSVCRT:gshandler.obj
 0001:00005da8       __GSHandlerCheckCommon     0000000180006da8 f   MSVCRT:gshandler.obj
 0001:00005e20       __security_check_cookie    0000000180006e20 f   MSVCRT:amdsecgs.obj
 0001:00006160       _DllMainCRTStartup         0000000180007160 f   MSVCRT:dll_dllmain.obj
 0001:000061a0       _guard_check_icall_nop     00000001800071a0 f i MSVCRT:guard_support.obj
 0001:000061a4       __raise_securityfailure    00000001800071a4 f   MSVCRT:gs_report.obj
 0001:000061d8       __report_gsfailure         00000001800071d8 f   MSVCRT:gs_report.obj
 0001:00006320       __security_init_cookie     0000000180007320 f   MSVCRT:gs_support.obj
 0001:000063cc       ?__scrt_initialize_type_info@@YAXXZ 00000001800073cc f   MSVCRT:tncleanup.obj
 0001:000063dc       ?__scrt_uninitialize_type_info@@YAXXZ 00000001800073dc f   MSVCRT:tncleanup.obj
 0001:000063e8       __scrt_initialize_default_local_stdio_options 00000001800073e8 f   MSVCRT:default_local_stdio_options.obj
 0001:00006404       __scrt_acquire_startup_lock 0000000180007404 f   MSVCRT:utility.obj
 0001:00006440       __scrt_dllmain_after_initialize_c 0000000180007440 f   MSVCRT:utility.obj
 0001:00006474       __scrt_dllmain_before_initialize_c 0000000180007474 f   MSVCRT:utility.obj
 0001:0000648c       __scrt_dllmain_crt_thread_attach 000000018000748c f   MSVCRT:utility.obj
 0001:000064b4       __scrt_dllmain_crt_thread_detach 00000001800074b4 f   MSVCRT:utility.obj
 0001:000064cc       __scrt_dllmain_exception_filter 00000001800074cc f   MSVCRT:utility.obj
 0001:0000652c       __scrt_dllmain_uninitialize_c 000000018000752c f   MSVCRT:utility.obj
 0001:0000655c       __scrt_dllmain_uninitialize_critical 000000018000755c f   MSVCRT:utility.obj
 0001:00006570       __scrt_initialize_crt      0000000180007570 f   MSVCRT:utility.obj
 0001:000065bc       __scrt_initialize_onexit_tables 00000001800075bc f   MSVCRT:utility.obj
 0001:00006648       __scrt_is_nonwritable_in_current_image 0000000180007648 f   MSVCRT:utility.obj
 0001:000066e0       __scrt_release_startup_lock 00000001800076e0 f   MSVCRT:utility.obj
 0001:00006704       __scrt_uninitialize_crt    0000000180007704 f   MSVCRT:utility.obj
 0001:00006730       __scrt_get_dyn_tls_init_callback 0000000180007730 f   MSVCRT:dyn_tls_init.obj
 0001:00006738       __crt_debugger_hook        0000000180007738 f   MSVCRT:utility_desktop.obj
 0001:00006740       __scrt_fastfail            0000000180007740 f   MSVCRT:utility_desktop.obj
 0001:0000688c       _RTC_Initialize            000000018000788c f   MSVCRT:initsect.obj
 0001:000068c8       _RTC_Terminate             00000001800078c8 f   MSVCRT:initsect.obj
 0001:00006910       __isa_available_init       0000000180007910 f   MSVCRT:cpu_disp.obj
 0001:00006abc       _get_startup_argv_mode     0000000180007abc f   MSVCRT:argv_mode.obj
 0001:00006ac4       __scrt_is_ucrt_dll_in_use  0000000180007ac4 f   MSVCRT:ucrt_detection.obj
 0001:00006ad0       memset                     0000000180007ad0 f   vcruntime:VCRUNTIME140.dll
 0001:00006ad6       wcschr                     0000000180007ad6 f   vcruntime:VCRUNTIME140.dll
 0001:00006adc       wcsstr                     0000000180007adc f   vcruntime:VCRUNTIME140.dll
 0001:00006ae2       memcpy                     0000000180007ae2 f   vcruntime:VCRUNTIME140.dll
 0001:00006ae8       __C_specific_handler       0000000180007ae8 f   vcruntime:VCRUNTIME140.dll
 0001:00006aee       __std_type_info_destroy_list 0000000180007aee f   vcruntime:VCRUNTIME140.dll
 0001:00006af4       strcpy                     0000000180007af4 f   ucrt:api-ms-win-crt-string-l1-1-0.dll
 0001:00006afa       strlen                     0000000180007afa f   ucrt:api-ms-win-crt-string-l1-1-0.dll
 0001:00006b00       strcat                     0000000180007b00 f   ucrt:api-ms-win-crt-string-l1-1-0.dll
 0001:00006b06       _initterm                  0000000180007b06 f   ucrt:api-ms-win-crt-runtime-l1-1-0.dll
 0001:00006b0c       _initterm_e                0000000180007b0c f   ucrt:api-ms-win-crt-runtime-l1-1-0.dll
 0001:00006b12       _seh_filter_dll            0000000180007b12 f   ucrt:api-ms-win-crt-runtime-l1-1-0.dll
 0001:00006b18       _configure_narrow_argv     0000000180007b18 f   ucrt:api-ms-win-crt-runtime-l1-1-0.dll
 0001:00006b1e       _initialize_narrow_environment 0000000180007b1e f   ucrt:api-ms-win-crt-runtime-l1-1-0.dll
 0001:00006b24       _initialize_onexit_table   0000000180007b24 f   ucrt:api-ms-win-crt-runtime-l1-1-0.dll
 0001:00006b2a       _execute_onexit_table      0000000180007b2a f   ucrt:api-ms-win-crt-runtime-l1-1-0.dll
 0001:00006b30       _cexit                     0000000180007b30 f   ucrt:api-ms-win-crt-runtime-l1-1-0.dll
 0001:00006b50       _guard_dispatch_icall_nop  0000000180007b50 f   MSVCRT:guard_dispatch.obj
 0001:00006b70       _guard_xfg_dispatch_icall_nop 0000000180007b70 f   MSVCRT:guard_xfg_dispatch.obj
 0002:00000000       __imp_RegCloseKey          0000000180008000     advapi32:ADVAPI32.dll
 0002:00000008       __imp_RegQueryValueExA     0000000180008008     advapi32:ADVAPI32.dll
 0002:00000010       __imp_RegOpenKeyExA        0000000180008010     advapi32:ADVAPI32.dll
 0002:00000018       \177ADVAPI32_NULL_THUNK_DATA 0000000180008018     advapi32:ADVAPI32.dll
 0002:00000020       __imp_TerminateProcess     0000000180008020     kernel32:KERNEL32.dll
 0002:00000028       __imp_GetCurrentProcess    0000000180008028     kernel32:KERNEL32.dll
 0002:00000030       __imp_SetUnhandledExceptionFilter 0000000180008030     kernel32:KERNEL32.dll
 0002:00000038       __imp_UnhandledExceptionFilter 0000000180008038     kernel32:KERNEL32.dll
 0002:00000040       __imp_RtlVirtualUnwind     0000000180008040     kernel32:KERNEL32.dll
 0002:00000048       __imp_RtlLookupFunctionEntry 0000000180008048     kernel32:KERNEL32.dll
 0002:00000050       __imp_RtlCaptureContext    0000000180008050     kernel32:KERNEL32.dll
 0002:00000058       __imp_LoadLibraryExA       0000000180008058     kernel32:KERNEL32.dll
 0002:00000060       __imp_GetModuleHandleW     0000000180008060     kernel32:KERNEL32.dll
 0002:00000068       __imp_FreeLibrary          0000000180008068     kernel32:KERNEL32.dll
 0002:00000070       __imp_VirtualProtect       0000000180008070     kernel32:KERNEL32.dll
 0002:00000078       __imp_QueryPerformanceCounter 0000000180008078     kernel32:KERNEL32.dll
 0002:00000080       __imp_GetLastError         0000000180008080     kernel32:KERNEL32.dll
 0002:00000088       __imp_RaiseException       0000000180008088     kernel32:KERNEL32.dll
 0002:00000090       __imp_VerifyVersionInfoW   0000000180008090     kernel32:KERNEL32.dll
 0002:00000098       __imp_SetHandleInformation 0000000180008098     kernel32:KERNEL32.dll
 0002:000000a0       __imp_VerSetConditionMask  00000001800080a0     kernel32:KERNEL32.dll
 0002:000000a8       __imp_WideCharToMultiByte  00000001800080a8     kernel32:KERNEL32.dll
 0002:000000b0       __imp_GetOverlappedResult  00000001800080b0     kernel32:KERNEL32.dll
 0002:000000b8       __imp_SetLastError         00000001800080b8     kernel32:KERNEL32.dll
 0002:000000c0       __imp_GetProcAddress       00000001800080c0     kernel32:KERNEL32.dll
 0002:000000c8       __imp_FormatMessageA       00000001800080c8     kernel32:KERNEL32.dll
 0002:000000d0       __imp_LocalFree            00000001800080d0     kernel32:KERNEL32.dll
 0002:000000d8       __imp_GlobalFree           00000001800080d8     kernel32:KERNEL32.dll
 0002:000000e0       __imp_IsProcessorFeaturePresent 00000001800080e0     kernel32:KERNEL32.dll
 0002:000000e8       __imp_GetCurrentProcessId  00000001800080e8     kernel32:KERNEL32.dll
 0002:000000f0       __imp_GetSystemInfo        00000001800080f0     kernel32:KERNEL32.dll
 0002:000000f8       __imp_VirtualQuery         00000001800080f8     kernel32:KERNEL32.dll
 0002:00000100       __imp_GetSystemTimeAsFileTime 0000000180008100     kernel32:KERNEL32.dll
 0002:00000108       __imp_InitializeSListHead  0000000180008108     kernel32:KERNEL32.dll
 0002:00000110       __imp_IsDebuggerPresent    0000000180008110     kernel32:KERNEL32.dll
 0002:00000118       __imp_GetCurrentThreadId   0000000180008118     kernel32:KERNEL32.dll
 0002:00000120       \177KERNEL32_NULL_THUNK_DATA 0000000180008120     kernel32:KERNEL32.dll
 0002:00000128       __imp_wcschr               0000000180008128     vcruntime:VCRUNTIME140.dll
 0002:00000130       __imp_wcsstr               0000000180008130     vcruntime:VCRUNTIME140.dll
 0002:00000138       __imp_memcpy               0000000180008138     vcruntime:VCRUNTIME140.dll
 0002:00000140       __imp___C_specific_handler 0000000180008140     vcruntime:VCRUNTIME140.dll
 0002:00000148       __imp_memset               0000000180008148     vcruntime:VCRUNTIME140.dll
 0002:00000150       __imp___std_type_info_destroy_list 0000000180008150     vcruntime:VCRUNTIME140.dll
 0002:00000158       \177VCRUNTIME140_NULL_THUNK_DATA 0000000180008158     vcruntime:VCRUNTIME140.dll
 0002:00000160       __imp_WinHttpGetIEProxyConfigForCurrentUser 0000000180008160     winhttp:WINHTTP.dll
 0002:00000168       __imp_WinHttpGetProxyForUrl 0000000180008168     winhttp:WINHTTP.dll
 0002:00000170       __imp_WinHttpOpen          0000000180008170     winhttp:WINHTTP.dll
 0002:00000178       \177WINHTTP_NULL_THUNK_DATA 0000000180008178     winhttp:WINHTTP.dll
 0002:00000180       __imp_WSACleanup           0000000180008180     ws2_32:WS2_32.dll
 0002:00000188       __imp_WSAStartup           0000000180008188     ws2_32:WS2_32.dll
 0002:00000190       __imp_socket               0000000180008190     ws2_32:WS2_32.dll
 0002:00000198       __imp_select               0000000180008198     ws2_32:WS2_32.dll
 0002:000001a0       __imp_WSASetLastError      00000001800081a0     ws2_32:WS2_32.dll
 0002:000001a8       __imp_WSAIoctl             00000001800081a8     ws2_32:WS2_32.dll
 0002:000001b0       __imp_ntohs                00000001800081b0     ws2_32:WS2_32.dll
 0002:000001b8       __imp_WSAAddressToStringA  00000001800081b8     ws2_32:WS2_32.dll
 0002:000001c0       __imp_getnameinfo          00000001800081c0     ws2_32:WS2_32.dll
 0002:000001c8       __imp_freeaddrinfo         00000001800081c8     ws2_32:WS2_32.dll
 0002:000001d0       __imp_bind                 00000001800081d0     ws2_32:WS2_32.dll
 0002:000001d8       __imp_getaddrinfo          00000001800081d8     ws2_32:WS2_32.dll
 0002:000001e0       __imp_WSAEventSelect       00000001800081e0     ws2_32:WS2_32.dll
 0002:000001e8       __imp_WSACreateEvent       00000001800081e8     ws2_32:WS2_32.dll
 0002:000001f0       __imp_WSACloseEvent        00000001800081f0     ws2_32:WS2_32.dll
 0002:000001f8       __imp_WSAGetLastError      00000001800081f8     ws2_32:WS2_32.dll
 0002:00000200       __imp_gethostname          0000000180008200     ws2_32:WS2_32.dll
 0002:00000208       __imp_setsockopt           0000000180008208     ws2_32:WS2_32.dll
 0002:00000210       __imp_ntohl                0000000180008210     ws2_32:WS2_32.dll
 0002:00000218       __imp_htons                0000000180008218     ws2_32:WS2_32.dll
 0002:00000220       __imp_htonl                0000000180008220     ws2_32:WS2_32.dll
 0002:00000228       __imp_getsockopt           0000000180008228     ws2_32:WS2_32.dll
 0002:00000230       __imp_connect              0000000180008230     ws2_32:WS2_32.dll
 0002:00000238       __imp_closesocket          0000000180008238     ws2_32:WS2_32.dll
 0002:00000240       __imp_ioctlsocket          0000000180008240     ws2_32:WS2_32.dll
 0002:00000248       \177WS2_32_NULL_THUNK_DATA 0000000180008248     ws2_32:WS2_32.dll
 0002:00000250       __imp_realloc              0000000180008250     ucrt:api-ms-win-crt-heap-l1-1-0.dll
 0002:00000258       __imp_free                 0000000180008258     ucrt:api-ms-win-crt-heap-l1-1-0.dll
 0002:00000260       __imp_malloc               0000000180008260     ucrt:api-ms-win-crt-heap-l1-1-0.dll
 0002:00000268       \177api-ms-win-crt-heap-l1-1-0_NULL_THUNK_DATA 0000000180008268     ucrt:api-ms-win-crt-heap-l1-1-0.dll
 0002:00000270       __imp__execute_onexit_table 0000000180008270     ucrt:api-ms-win-crt-runtime-l1-1-0.dll
 0002:00000278       __imp__initialize_onexit_table 0000000180008278     ucrt:api-ms-win-crt-runtime-l1-1-0.dll
 0002:00000280       __imp__initialize_narrow_environment 0000000180008280     ucrt:api-ms-win-crt-runtime-l1-1-0.dll
 0002:00000288       __imp__configure_narrow_argv 0000000180008288     ucrt:api-ms-win-crt-runtime-l1-1-0.dll
 0002:00000290       __imp__seh_filter_dll      0000000180008290     ucrt:api-ms-win-crt-runtime-l1-1-0.dll
 0002:00000298       __imp__initterm            0000000180008298     ucrt:api-ms-win-crt-runtime-l1-1-0.dll
 0002:000002a0       __imp__errno               00000001800082a0     ucrt:api-ms-win-crt-runtime-l1-1-0.dll
 0002:000002a8       __imp__cexit               00000001800082a8     ucrt:api-ms-win-crt-runtime-l1-1-0.dll
 0002:000002b0       __imp__initterm_e          00000001800082b0     ucrt:api-ms-win-crt-runtime-l1-1-0.dll
 0002:000002b8       \177api-ms-win-crt-runtime-l1-1-0_NULL_THUNK_DATA 00000001800082b8     ucrt:api-ms-win-crt-runtime-l1-1-0.dll
 0002:000002c0       __imp___stdio_common_vswscanf 00000001800082c0     ucrt:api-ms-win-crt-stdio-l1-1-0.dll
 0002:000002c8       __imp___stdio_common_vsprintf 00000001800082c8     ucrt:api-ms-win-crt-stdio-l1-1-0.dll
 0002:000002d0       __imp___stdio_common_vswprintf 00000001800082d0     ucrt:api-ms-win-crt-stdio-l1-1-0.dll
 0002:000002d8       \177api-ms-win-crt-stdio-l1-1-0_NULL_THUNK_DATA 00000001800082d8     ucrt:api-ms-win-crt-stdio-l1-1-0.dll
 0002:000002e0       __imp_strcat               00000001800082e0     ucrt:api-ms-win-crt-string-l1-1-0.dll
 0002:000002e8       __imp_strcpy               00000001800082e8     ucrt:api-ms-win-crt-string-l1-1-0.dll
 0002:000002f0       __imp_wcslen               00000001800082f0     ucrt:api-ms-win-crt-string-l1-1-0.dll
 0002:000002f8       __imp_wcsncmp              00000001800082f8     ucrt:api-ms-win-crt-string-l1-1-0.dll
 0002:00000300       __imp_wcstok_s             0000000180008300     ucrt:api-ms-win-crt-string-l1-1-0.dll
 0002:00000308       __imp__wcsdup              0000000180008308     ucrt:api-ms-win-crt-string-l1-1-0.dll
 0002:00000310       __imp_strlen               0000000180008310     ucrt:api-ms-win-crt-string-l1-1-0.dll
 0002:00000318       __imp_wcscmp               0000000180008318     ucrt:api-ms-win-crt-string-l1-1-0.dll
 0002:00000320       \177api-ms-win-crt-string-l1-1-0_NULL_THUNK_DATA 0000000180008320     ucrt:api-ms-win-crt-string-l1-1-0.dll
 0002:00000328       __imp_JNU_ThrowByNameWithMessageAndLastError 0000000180008328     java:java.dll
 0002:00000330       __imp_JNU_ThrowInternalError 0000000180008330     java:java.dll
 0002:00000338       __imp_JNU_ThrowOutOfMemoryError 0000000180008338     java:java.dll
 0002:00000340       __imp_JNU_ThrowByName      0000000180008340     java:java.dll
 0002:00000348       __imp_JNU_ThrowNullPointerException 0000000180008348     java:java.dll
 0002:00000350       __imp_JNU_NewStringPlatform 0000000180008350     java:java.dll
 0002:00000358       __imp_JDK_LoadSystemLibrary 0000000180008358     java:java.dll
 0002:00000360       __imp_JNU_ReleaseStringPlatformChars 0000000180008360     java:java.dll
 0002:00000368       __imp_JNU_GetStringPlatformCharsStrict 0000000180008368     java:java.dll
 0002:00000370       \177java_NULL_THUNK_DATA   0000000180008370     java:java.dll
 0002:00000378       __imp_JVM_CurrentTimeMillis 0000000180008378     jvm:jvm.dll
 0002:00000380       __imp_jio_snprintf         0000000180008380     jvm:jvm.dll
 0002:00000388       \177jvm_NULL_THUNK_DATA    0000000180008388     jvm:jvm.dll
 0002:00000390       __guard_check_icall_fptr   0000000180008390     MSVCRT:guard_support.obj
 0002:00000398       __guard_xfg_check_icall_fptr 0000000180008398     MSVCRT:guard_support.obj
 0002:000003a0       __guard_dispatch_icall_fptr 00000001800083a0     MSVCRT:guard_support.obj
 0002:000003a8       __guard_xfg_dispatch_icall_fptr 00000001800083a8     MSVCRT:guard_support.obj
 0002:000003b0       __guard_xfg_table_dispatch_icall_fptr 00000001800083b0     MSVCRT:guard_support.obj
 0002:000003b8       __castguard_check_failure_os_handled_fptr 00000001800083b8     MSVCRT:guard_support.obj
 0002:000003c0       __guard_memcpy_fptr        00000001800083c0     vcruntime:softmemtag.obj
 0002:000003c8       __xc_a                     00000001800083c8     MSVCRT:initializers.obj
 0002:000003d0       __xc_z                     00000001800083d0     MSVCRT:initializers.obj
 0002:000003d8       __xi_a                     00000001800083d8     MSVCRT:initializers.obj
 0002:000003e0       __xi_z                     00000001800083e0     MSVCRT:initializers.obj
 0002:000003e8       __xp_a                     00000001800083e8     MSVCRT:initializers.obj
 0002:000003f0       __xp_z                     00000001800083f0     MSVCRT:initializers.obj
 0002:000003f8       __xt_a                     00000001800083f8     MSVCRT:initializers.obj
 0002:00000400       __xt_z                     0000000180008400     MSVCRT:initializers.obj
 0002:00000420       ??_C@_1CG@FPLLFFJC@?$AAO?$AAn?$AAl?$AAy?$AA?5?$AAu?$AAs?$AAe?$AAd?$AA?5?$AAi?$AAn?$AAt?$AAe?$AAr@ 0000000180008420     DefaultProxySelector.obj
 0002:00000448       ??_C@_17IAHLGHKI@?$AA?3?$AA?1?$AA?1@ 0000000180008448     DefaultProxySelector.obj
 0002:00000450       ??_C@_15KNBIKKIN@?$AA?$CF?$AAd@ 0000000180008450     DefaultProxySelector.obj
 0002:00000458       ??_C@_1BA@KGNJOJGK@?$AA?$CF?$AAs?$AA?3?$AA?1?$AA?1?$AA?$CF?$AAs@ 0000000180008458     DefaultProxySelector.obj
 0002:00000468       ??_C@_15IALCAGAM@?$AA?$DL?$AA?5@ 0000000180008468     DefaultProxySelector.obj
 0002:00000470       ??_C@_1BA@PAMDJABJ@?$AA?$DM?$AAl?$AAo?$AAc?$AAa?$AAl?$AA?$DO@ 0000000180008470     DefaultProxySelector.obj
 0002:00000480       ??_C@_19NNDKDCM@?$AAh?$AAt?$AAt?$AAp@ 0000000180008480     DefaultProxySelector.obj
 0002:00000490       ??_C@_17HHNFGGOB@?$AAf?$AAt?$AAp@ 0000000180008490     DefaultProxySelector.obj
 0002:00000498       ??_C@_1M@PGEJLFN@?$AAh?$AAt?$AAt?$AAp?$AAs@ 0000000180008498     DefaultProxySelector.obj
 0002:000004a8       ??_C@_1M@LCMPGCNK@?$AAs?$AAo?$AAc?$AAk?$AAs@ 00000001800084a8     DefaultProxySelector.obj
 0002:000004b8       ??_C@_0BG@MGDLLCGN@java?1net?1Inet4Address@ 00000001800084b8     Inet4Address.obj
 0002:000004d0       ??_C@_03GAEACAIP@?$CI?$CJV@ 00000001800084d0     Inet4Address.obj
 0002:000004d4       ??_C@_06FALKBLGB@?$DMinit?$DO@ 00000001800084d4     Inet4Address.obj
 0002:000004e0       ??_C@_09IPAEKDAI@localhost@ 00000001800084e0     Inet4AddressImpl.obj
 0002:000004f0       ??_C@_0BG@FFLEOBNG@host?5argument?5is?5null@ 00000001800084f0     Inet4AddressImpl.obj
 0002:00000508       ??_C@_0BO@JEDADEEB@java?1net?1UnknownHostException@ 0000000180008508     Inet4AddressImpl.obj
 0002:00000528       ??_C@_0BO@IKFIAFAI@Native?5heap?5allocation?5failed@ 0000000180008528     Inet4AddressImpl.obj
 0002:00000548       ??_C@_0BE@KNBHMLLP@Can?8t?5create?5socket@ 0000000180008548     Inet4AddressImpl.obj
 0002:00000560       ??_C@_0BC@LNOJFPHG@Can?8t?5bind?5socket@ 0000000180008560     Inet4AddressImpl.obj
 0002:00000578       ??_C@_0P@FKKLKLOM@connect?5failed@ 0000000180008578     Inet4AddressImpl.obj
 0002:00000588       ??_C@_0BK@LKDLOIJL@java?1net?1ConnectException@ 0000000180008588     Inet4AddressImpl.obj
 0002:000005a8       ??_C@_0BK@CJOLIFJC@Unable?5to?5allocate?5memory@ 00000001800085a8     Inet4AddressImpl.obj
 0002:000005c8       ??_C@_0CC@EAIDNHEI@Unable?5to?5create?5ICMP?5file?5hand@ 00000001800085c8     Inet4AddressImpl.obj
 0002:000005f0       ??_C@_0BG@OIMNJKOL@java?1net?1Inet6Address@ 00000001800085f0     Inet6Address.obj
 0002:00000608       ??_C@_0CJ@HANKHEO@java?1net?1Inet6Address$Inet6Addr@ 0000000180008608     Inet6Address.obj
 0002:00000638       ??_C@_0CL@OGPDIPGP@Ljava?1net?1Inet6Address$Inet6Add@ 0000000180008638     Inet6Address.obj
 0002:00000668       ??_C@_07CFDIJDEC@holder6@  0000000180008668     Inet6Address.obj
 0002:00000670       ??_C@_02KCBIMKDL@?$FLB@    0000000180008670     Inet6Address.obj
 0002:00000678       ??_C@_09OMLGLGNL@ipaddress@ 0000000180008678     Inet6Address.obj
 0002:00000684       ??_C@_01JPJNBJEM@I@        0000000180008684     Inet6Address.obj
 0002:00000688       ??_C@_08HMELDLBB@scope_id@ 0000000180008688     Inet6Address.obj
 0002:00000694       ??_C@_01POHCFINO@Z@        0000000180008694     Inet6Address.obj
 0002:00000698       ??_C@_0N@EMCDHDAD@scope_id_set@ 0000000180008698     Inet6Address.obj
 0002:000006a8       ??_C@_0BM@MEIIMOAC@Ljava?1net?1NetworkInterface?$DL@ 00000001800086a8     Inet6Address.obj
 0002:000006c8       ??_C@_0N@DKHAKOIC@scope_ifname@ 00000001800086c8     Inet6Address.obj
 0002:000006d8       ??_C@_0BP@NBCDDEJF@Can?8t?5bind?5socket?5to?5interface@ 00000001800086d8     Inet6AddressImpl.obj
 0002:000006f8       ??_C@_0BF@LNJHKELF@java?1net?1InetAddress@ 00000001800086f8     InetAddress.obj
 0002:00000710       ??_C@_0CH@OBMJDEDM@java?1net?1InetAddress$InetAddres@ 0000000180008710     InetAddress.obj
 0002:00000738       ??_C@_0CJ@BPCMNDLL@Ljava?1net?1InetAddress$InetAddre@ 0000000180008738     InetAddress.obj
 0002:00000764       ??_C@_06JIPLHHCL@holder@   0000000180008764     InetAddress.obj
 0002:00000770       ??_C@_07LHEPONKL@address@  0000000180008770     InetAddress.obj
 0002:00000778       ??_C@_06NBOBHOCP@family@   0000000180008778     InetAddress.obj
 0002:00000780       ??_C@_0BD@JFADHEFE@Ljava?1lang?1String?$DL@ 0000000180008780     InetAddress.obj
 0002:00000798       ??_C@_08IGGJEOEE@hostName@ 0000000180008798     InetAddress.obj
 0002:000007a8       ??_C@_0BB@JAHGOJG@originalHostName@ 00000001800087a8     InetAddress.obj
 0002:000007bc       ??_C@_01LELAEKIP@J@        00000001800087bc     NTLMAuthSequence.obj
 0002:000007c0       ??_C@_09ILBCNDDJ@ctxHandle@ 00000001800087c0     NTLMAuthSequence.obj
 0002:000007d0       ??_C@_09NDBMIONH@crdHandle@ 00000001800087d0     NTLMAuthSequence.obj
 0002:000007e0       ??_C@_0BB@KLNFJBDM@sequenceComplete@ 00000001800087e0     NTLMAuthSequence.obj
 0002:000007f8       ??_C@_0CA@NIIGFDJD@native?5memory?5allocation?5failed@ 00000001800087f8     NTLMAuthSequence.obj
 0002:00000818       ??_C@_04KGCGDDND@NTLM@     0000000180008818     NTLMAuthSequence.obj
 0002:00000820       ??_C@_0L@BFDIJHCF@urlmon?4dll@ 0000000180008820     NTLMAuthentication.obj
 0002:00000830       ??_C@_0CA@OOMLPODH@CoInternetCreateSecurityManager@ 0000000180008830     NTLMAuthentication.obj
 0002:00000850       ??_C@_0BJ@PLKHNKJH@GetUnicastIpAddressTable@ 0000000180008850     NetworkInterface.obj
 0002:00000870       ??_C@_0BJ@IJNLNPKI@java?1net?1SocketException@ 0000000180008870     NetworkInterface.obj
 0002:00000890       ??_C@_0BJ@OODHKIPD@GetAnycastIpAddressTable@ 0000000180008890     NetworkInterface.obj
 0002:000008b0       ??_C@_0BM@JKGHLHKJ@ConvertInterfaceLuidToNameW@ 00000001800088b0     NetworkInterface.obj
 0002:000008d0       ??_C@_0M@KMPMMAFM@native?5heap@ 00000001800088d0     NetworkInterface.obj
 0002:000008e0       ??_C@_0BI@ICICOKAH@ConvertLengthToIpv4Mask@ 00000001800088e0     NetworkInterface.obj
 0002:000008f8       ??_C@_0M@CFLMHJFF@GetIfEntry2@ 00000001800088f8     NetworkInterface.obj
 0002:00000908       ??_C@_0BM@CAOLEHGP@ConvertInterfaceNameToLuidW@ 0000000180008908     NetworkInterface.obj
 0002:00000928       ??_C@_0M@FPBJEEGA@GetIfTable2@ 0000000180008928     NetworkInterface.obj
 0002:00000934       ??_C@_04MEMAJGDJ@name@     0000000180008934     NetworkInterface.obj
 0002:00000940       ??_C@_0M@NDEOCEGH@displayName@ 0000000180008940     NetworkInterface.obj
 0002:0000094c       ??_C@_05FKHKFDID@index@    000000018000894c     NetworkInterface.obj
 0002:00000958       ??_C@_0BI@FKGHKPME@?$FLLjava?1net?1InetAddress?$DL@ 0000000180008958     NetworkInterface.obj
 0002:00000970       ??_C@_05GAEKFHB@addrs@     0000000180008970     NetworkInterface.obj
 0002:00000978       ??_C@_0BN@FGCEFHCI@?$FLLjava?1net?1InterfaceAddress?$DL@ 0000000180008978     NetworkInterface.obj
 0002:00000998       ??_C@_08OKHKOBIL@bindings@ 0000000180008998     NetworkInterface.obj
 0002:000009a8       ??_C@_0BN@LEABGBNB@?$FLLjava?1net?1NetworkInterface?$DL@ 00000001800089a8     NetworkInterface.obj
 0002:000009c8       ??_C@_06JCHEOPIA@childs@   00000001800089c8     NetworkInterface.obj
 0002:000009d0       ??_C@_0BK@HBDFEEEP@java?1net?1InterfaceAddress@ 00000001800089d0     NetworkInterface.obj
 0002:000009f0       ??_C@_0BH@FIKCFBLO@Ljava?1net?1InetAddress?$DL@ 00000001800089f0     NetworkInterface.obj
 0002:00000a08       ??_C@_0BI@EDMBHPFP@Ljava?1net?1Inet4Address?$DL@ 0000000180008a08     NetworkInterface.obj
 0002:00000a20       ??_C@_09OALBOHJN@broadcast@ 0000000180008a20     NetworkInterface.obj
 0002:00000a2c       ??_C@_01CPLAODJH@S@        0000000180008a2c     NetworkInterface.obj
 0002:00000a30       ??_C@_0L@NAAPBPMO@maskLength@ 0000000180008a30     NetworkInterface.obj
 0002:00000a40       ??_C@_0BP@FOGJMHII@Native?5heap?5allocation?5failure@ 0000000180008a40     ResolverConfigurationImpl.obj
 0002:00000a60       ??_C@_0BL@ENCPOIKC@java?1lang?1OutOfMemoryError@ 0000000180008a60     ResolverConfigurationImpl.obj
 0002:00000a80       ??_C@_0EK@CCGONJEN@IP?5Helper?5Library?5GetAdaptersAd@ 0000000180008a80     ResolverConfigurationImpl.obj
 0002:00000ad0       ??_C@_0EK@DMMHGOF@IP?5Helper?5Library?5GetAdaptersAd@ 0000000180008ad0     ResolverConfigurationImpl.obj
 0002:00000b20       ??_C@_0DH@HIDBKCBL@IP?5Helper?5Library?5GetAdaptersAd@ 0000000180008b20     ResolverConfigurationImpl.obj
 0002:00000b58       ??_C@_01IHBHIGKO@?0@       0000000180008b58     ResolverConfigurationImpl.obj
 0002:00000b60       ??_C@_0DD@IKBMIFKO@SYSTEM?2CurrentControlSet?2Servic@ 0000000180008b60     ResolverConfigurationImpl.obj
 0002:00000b98       ??_C@_0L@HPLHIFHN@SearchList@ 0000000180008b98     ResolverConfigurationImpl.obj
 0002:00000ba8       ??_C@_0O@BBEOADGN@os_searchlist@ 0000000180008ba8     ResolverConfigurationImpl.obj
 0002:00000bb8       ??_C@_0P@HAAMGONH@os_nameservers@ 0000000180008bb8     ResolverConfigurationImpl.obj
 0002:00000bc8       ??_C@_0BC@DDPBLLCP@java?1lang?1Boolean@ 0000000180008bc8     net_util.obj
 0002:00000be0       ??_C@_0BG@CGIGLAGP@?$CILjava?1lang?1String?$DL?$CJZ@ 0000000180008be0     net_util.obj
 0002:00000bf8       ??_C@_0L@HKKDKOBF@getBoolean@ 0000000180008bf8     net_util.obj
 0002:00000c08       ??_C@_0BJ@OCGKBLBN@java?4net?4preferIPv4Stack@ 0000000180008c08     net_util.obj
 0002:00000c28       ??_C@_0BL@KNKNLGPI@InetAddress?5holder?5is?5null@ 0000000180008c28     net_util.obj
 0002:00001088       ??_C@_0BC@HFNFNKAI@Permission?5denied@ 0000000180009088     net_util_md.obj
 0002:000010a0       ??_C@_0O@GLDCGPDO@BindException@ 00000001800090a0     net_util_md.obj
 0002:000010b0       ??_C@_0BH@LOKACPE@Address?5already?5in?5use@ 00000001800090b0     net_util_md.obj
 0002:000010c8       ??_C@_0CA@NBHADPNL@Cannot?5assign?5requested?5address@ 00000001800090c8     net_util_md.obj
 0002:000010e8       ??_C@_0DA@KDGLCJJO@Address?5family?5not?5supported?5by@ 00000001800090e8     net_util_md.obj
 0002:00001118       ??_C@_0BO@BMABNIPB@Operation?5already?5in?5progress@ 0000000180009118     net_util_md.obj
 0002:00001138       ??_C@_0CB@DJAOADN@Software?5caused?5connection?5abor@ 0000000180009138     net_util_md.obj
 0002:00001160       ??_C@_0BB@CICOPLDE@ConnectException@ 0000000180009160     net_util_md.obj
 0002:00001178       ??_C@_0BD@NPDMPPFP@Connection?5refused@ 0000000180009178     net_util_md.obj
 0002:00001190       ??_C@_0BJ@FJAMCHKE@Connection?5reset?5by?5peer@ 0000000180009190     net_util_md.obj
 0002:000011b0       ??_C@_0BN@HFCIEIME@Destination?5address?5required@ 00000001800091b0     net_util_md.obj
 0002:000011d0       ??_C@_0M@LOEHLCJD@Bad?5address@ 00000001800091d0     net_util_md.obj
 0002:000011e0       ??_C@_0N@OHOPOBEF@Host?5is?5down@ 00000001800091e0     net_util_md.obj
 0002:000011f0       ??_C@_0BH@PBADJGIL@NoRouteToHostException@ 00000001800091f0     net_util_md.obj
 0002:00001208       ??_C@_0BB@PFBILCPA@No?5route?5to?5host@ 0000000180009208     net_util_md.obj
 0002:00001220       ??_C@_0BK@LBMNDGCG@Operation?5now?5in?5progress@ 0000000180009220     net_util_md.obj
 0002:00001240       ??_C@_0BK@FJBOAFDK@Interrupted?5function?5call@ 0000000180009240     net_util_md.obj
 0002:00001260       ??_C@_0BB@HMGGCEBG@Invalid?5argument@ 0000000180009260     net_util_md.obj
 0002:00001278       ??_C@_0BM@CCONNCKE@Socket?5is?5already?5connected@ 0000000180009278     net_util_md.obj
 0002:00001298       ??_C@_0BE@INBJMKGG@Too?5many?5open?5files@ 0000000180009298     net_util_md.obj
 0002:000012b0       ??_C@_0EN@MMGGBIMI@The?5message?5is?5larger?5than?5the?5@ 00000001800092b0     net_util_md.obj
 0002:00001300       ??_C@_0BA@LPIEBGEK@Network?5is?5down@ 0000000180009300     net_util_md.obj
 0002:00001310       ??_C@_0CE@JHDCOCF@Network?5dropped?5connection?5on?5r@ 0000000180009310     net_util_md.obj
 0002:00001338       ??_C@_0BH@CIEOBPFM@Network?5is?5unreachable@ 0000000180009338     net_util_md.obj
 0002:00001350       ??_C@_0DJ@FJOKEEBP@No?5buffer?5space?5available?5?$CImaxi@ 0000000180009350     net_util_md.obj
 0002:00001390       ??_C@_0BE@NEGCDJON@Bad?5protocol?5option@ 0000000180009390     net_util_md.obj
 0002:000013a8       ??_C@_0BI@ILAOGBJJ@Socket?5is?5not?5connected@ 00000001800093a8     net_util_md.obj
 0002:000013c0       ??_C@_0BO@PFGGHOGH@Socket?5operation?5on?5nonsocket@ 00000001800093c0     net_util_md.obj
 0002:000013e0       ??_C@_0BI@EDJAHLMH@Operation?5not?5supported@ 00000001800093e0     net_util_md.obj
 0002:000013f8       ??_C@_0BO@EBCCBLCJ@Protocol?5family?5not?5supported@ 00000001800093f8     net_util_md.obj
 0002:00001418       ??_C@_0BD@LPHIGPM@Too?5many?5processes@ 0000000180009418     net_util_md.obj
 0002:00001430       ??_C@_0BH@JNBKLLAJ@Protocol?5not?5supported@ 0000000180009430     net_util_md.obj
 0002:00001448       ??_C@_0BP@PDKJLOAE@Protocol?5wrong?5type?5for?5socket@ 0000000180009448     net_util_md.obj
 0002:00001468       ??_C@_0CC@DAIJOIKC@Cannot?5send?5after?5socket?5shutdo@ 0000000180009468     net_util_md.obj
 0002:00001490       ??_C@_0BK@LMAIHBL@Socket?5type?5not?5supported@ 0000000180009490     net_util_md.obj
 0002:000014b0       ??_C@_0BF@IBBHAGLD@Connection?5timed?5out@ 00000001800094b0     net_util_md.obj
 0002:000014c8       ??_C@_0BF@EHICFGGJ@Class?5type?5not?5found@ 00000001800094c8     net_util_md.obj
 0002:000014e0       ??_C@_0CB@EPFKGNAK@Resource?5temporarily?5unavailabl@ 00000001800094e0     net_util_md.obj
 0002:00001508       ??_C@_0P@CAFMJNJH@Host?5not?5found@ 0000000180009508     net_util_md.obj
 0002:00001518       ??_C@_0BO@GICNLCFB@Insufficient?5memory?5available@ 0000000180009518     net_util_md.obj
 0002:00001538       ??_C@_0CI@CFJNLLNI@Successful?5WSAStartup?5not?5yet?5p@ 0000000180009538     net_util_md.obj
 0002:00001560       ??_C@_0CN@KFPNHBIN@Valid?5name?0?5no?5data?5record?5of?5r@ 0000000180009560     net_util_md.obj
 0002:00001590       ??_C@_0BP@BOOHLDLA@This?5is?5a?5nonrecoverable?5error@ 0000000180009590     net_util_md.obj
 0002:000015b0       ??_C@_0CB@PLJNFILF@Network?5subsystem?5is?5unavailabl@ 00000001800095b0     net_util_md.obj
 0002:000015d8       ??_C@_0CA@DOKOCCFB@Nonauthoritative?5host?5not?5found@ 00000001800095d8     net_util_md.obj
 0002:000015f8       ??_C@_0CB@GHMLGJBG@Winsock?4dll?5version?5out?5of?5rang@ 00000001800095f8     net_util_md.obj
 0002:00001620       ??_C@_0BO@ILFFGILJ@Graceful?5shutdown?5in?5progress@ 0000000180009620     net_util_md.obj
 0002:00001640       ??_C@_0BN@KGMIDOOK@Overlapped?5operation?5aborted@ 0000000180009640     net_util_md.obj
 0002:00001660       ??_C@_0BH@GDIHDDN@no?5further?5information@ 0000000180009660     net_util_md.obj
 0002:00001678       ??_C@_06DJHOIPC@?$CFs?3?5?$CFs@ 0000000180009678     net_util_md.obj
 0002:00001680       ??_C@_0CL@EIMGMHJP@Unrecognized?5Windows?5Sockets?5er@ 0000000180009680     net_util_md.obj
 0002:000016b0       ??_C@_0BA@EOEGOLGE@SocketException@ 00000001800096b0     net_util_md.obj
 0002:000016c0       ??_C@_09ELLCMIIO@java?1net?1@ 00000001800096c0     net_util_md.obj
 0002:000016cc       ??_C@_04HDOCAJNK@?$CFs?$CFs@ 00000001800096cc     net_util_md.obj
 0002:000016d8       ??_C@_0BM@PJBFLPGI@Protocol?5family?5unavailable@ 00000001800096d8     net_util_md.obj
 0002:000016f8       ??_C@_0P@CALONDPA@java?1net?1Proxy@ 00000001800096f8     proxy_util.obj
 0002:00001708       ??_C@_0DB@PIODMB@?$CILjava?1net?1Proxy$Type?$DLLjava?1net@ 0000000180009708     proxy_util.obj
 0002:00001740       ??_C@_0BE@CNHDIHBN@java?1net?1Proxy$Type@ 0000000180009740     proxy_util.obj
 0002:00001758       ??_C@_0BG@JJBIBCMK@Ljava?1net?1Proxy$Type?$DL@ 0000000180009758     proxy_util.obj
 0002:00001770       ??_C@_04MEDPFIKH@HTTP@     0000000180009770     proxy_util.obj
 0002:00001778       ??_C@_05HKHMHAPI@SOCKS@    0000000180009778     proxy_util.obj
 0002:00001780       ??_C@_0BB@GMCFBELK@Ljava?1net?1Proxy?$DL@ 0000000180009780     proxy_util.obj
 0002:00001798       ??_C@_08KOHKDPPJ@NO_PROXY@ 0000000180009798     proxy_util.obj
 0002:000017a8       ??_C@_0BL@HBNNAPLM@java?1net?1InetSocketAddress@ 00000001800097a8     proxy_util.obj
 0002:000017c8       ??_C@_0DC@FDHLAKNF@?$CILjava?1lang?1String?$DLI?$CJLjava?1net?1@ 00000001800097c8     proxy_util.obj
 0002:00001800       ??_C@_0BB@BNNOLJPL@createUnresolved@ 0000000180009800     proxy_util.obj
 0002:00001818       in6addr_any                0000000180009818     ws2_32:indef.obj
 0002:00001830       __sz_Secur32_dll           0000000180009830     secur32:Secur32.dll
 0002:00001840       __sz_IPHLPAPI_DLL          0000000180009840     iphlpapi:IPHLPAPI.DLL
 0002:00001850       ??_C@_1BK@DBDEIDLH@?$AAK?$AAE?$AAR?$AAN?$AAE?$AAL?$AA3?$AA2?$AA?4?$AAD?$AAL?$AAL@ 0000000180009850     delayimp:delayhlp.obj
 0002:00001870       ??_C@_0BI@OMNLIJDB@AcquireSRWLockExclusive@ 0000000180009870     delayimp:delayhlp.obj
 0002:00001888       ??_C@_0BI@HMIEPCNJ@ReleaseSRWLockExclusive@ 0000000180009888     delayimp:delayhlp.obj
 0002:000018a0       __pfnDliNotifyHook2        00000001800098a0     delayimp:delayhk2.obj
 0002:000018a8       __pfnDliFailureHook2       00000001800098a8     delayimp:delayhk1.obj
 0002:000018b0       _pDefaultRawDllMain        00000001800098b0     MSVCRT:dll_dllmain.obj
 0002:000018b0       _pRawDllMain               00000001800098b0     MSVCRT:dll_dllmain.obj
 0002:000018c0       _load_config_used          00000001800098c0     MSVCRT:loadcfg.obj
 0002:00001a10       __xmm@ffffffffffffffffffffffffffffffff 0000000180009a10     MSVCRT:utility.obj
 0002:00001b00       __volatile_metadata        0000000180009b00     <linker-defined>
 0002:00001ec0       __rtc_iaa                  0000000180009ec0     MSVCRT:initsect.obj
 0002:00001ec8       __rtc_izz                  0000000180009ec8     MSVCRT:initsect.obj
 0002:00001ed0       __rtc_taa                  0000000180009ed0     MSVCRT:initsect.obj
 0002:00001ed8       __rtc_tzz                  0000000180009ed8     MSVCRT:initsect.obj
 0002:00002484       __DELAY_IMPORT_DESCRIPTOR_secur32_dll 000000018000a484     secur32:Secur32.dll
 0002:000024a4       __DELAY_IMPORT_DESCRIPTOR_iphlpapi_dll 000000018000a4a4     iphlpapi:IPHLPAPI.DLL
 0002:000024c4       __NULL_DELAY_IMPORT_DESCRIPTOR 000000018000a4c4     secur32:Secur32.dll
 0002:00002568       \177IPHLPAPI_NULL_THUNK_DATA_DLN 000000018000a568     iphlpapi:IPHLPAPI.DLL
 0002:00002598       \177Secur32_NULL_THUNK_DATA_DLN 000000018000a598     secur32:Secur32.dll
 0002:00002778       \177Secur32_NULL_THUNK_DATA_DLB 000000018000a778     secur32:Secur32.dll
 0002:000027a8       \177IPHLPAPI_NULL_THUNK_DATA_DLB 000000018000a7a8     iphlpapi:IPHLPAPI.DLL
 0002:0000327c       __IMPORT_DESCRIPTOR_WS2_32 000000018000b27c     ws2_32:WS2_32.dll
 0002:00003290       __IMPORT_DESCRIPTOR_jvm    000000018000b290     jvm:jvm.dll
 0002:000032a4       __IMPORT_DESCRIPTOR_WINHTTP 000000018000b2a4     winhttp:WINHTTP.dll
 0002:000032b8       __IMPORT_DESCRIPTOR_java   000000018000b2b8     java:java.dll
 0002:000032cc       __IMPORT_DESCRIPTOR_ADVAPI32 000000018000b2cc     advapi32:ADVAPI32.dll
 0002:000032e0       __IMPORT_DESCRIPTOR_KERNEL32 000000018000b2e0     kernel32:KERNEL32.dll
 0002:000032f4       __IMPORT_DESCRIPTOR_VCRUNTIME140 000000018000b2f4     vcruntime:VCRUNTIME140.dll
 0002:00003308       __IMPORT_DESCRIPTOR_api-ms-win-crt-string-l1-1-0 000000018000b308     ucrt:api-ms-win-crt-string-l1-1-0.dll
 0002:0000331c       __IMPORT_DESCRIPTOR_api-ms-win-crt-stdio-l1-1-0 000000018000b31c     ucrt:api-ms-win-crt-stdio-l1-1-0.dll
 0002:00003330       __IMPORT_DESCRIPTOR_api-ms-win-crt-heap-l1-1-0 000000018000b330     ucrt:api-ms-win-crt-heap-l1-1-0.dll
 0002:00003344       __IMPORT_DESCRIPTOR_api-ms-win-crt-runtime-l1-1-0 000000018000b344     ucrt:api-ms-win-crt-runtime-l1-1-0.dll
 0002:00003358       __NULL_IMPORT_DESCRIPTOR   000000018000b358     ws2_32:WS2_32.dll
 0003:00000000       isRcvTimeoutSupported      000000018000c000     net_util_md.obj
 0003:000000a0       __security_cookie_complement 000000018000c0a0     MSVCRT:gs_cookie.obj
 0003:000000a8       __security_cookie          000000018000c0a8     MSVCRT:gs_cookie.obj
 0003:000000b0       __scrt_native_dllmain_reason 000000018000c0b0     MSVCRT:utility.obj
 0003:000000c0       __isa_available            000000018000c0c0     MSVCRT:cpu_disp.obj
 0003:000000c4       __isa_enabled              000000018000c0c4     MSVCRT:cpu_disp.obj
 0003:000000c8       __memset_fast_string_threshold 000000018000c0c8     MSVCRT:cpu_disp.obj
 0003:000000d0       __memset_nt_threshold      000000018000c0d0     MSVCRT:cpu_disp.obj
 0003:000000d8       __scrt_ucrt_dll_is_in_use  000000018000c0d8     MSVCRT:ucrt_stubs.obj
 0003:000000e0       __imp_Icmp6CreateFile      000000018000c0e0     iphlpapi:IPHLPAPI.DLL
 0003:000000e8       __imp_NotifyAddrChange     000000018000c0e8     iphlpapi:IPHLPAPI.DLL
 0003:000000f0       __imp_ConvertLengthToIpv4Mask 000000018000c0f0     iphlpapi:IPHLPAPI.DLL
 0003:000000f8       __imp_ConvertInterfaceLuidToNameW 000000018000c0f8     iphlpapi:IPHLPAPI.DLL
 0003:00000100       __imp_ConvertInterfaceNameToLuidW 000000018000c100     iphlpapi:IPHLPAPI.DLL
 0003:00000108       __imp_FreeMibTable         000000018000c108     iphlpapi:IPHLPAPI.DLL
 0003:00000110       __imp_IcmpCreateFile       000000018000c110     iphlpapi:IPHLPAPI.DLL
 0003:00000118       __imp_GetAnycastIpAddressTable 000000018000c118     iphlpapi:IPHLPAPI.DLL
 0003:00000120       __imp_IcmpCloseHandle      000000018000c120     iphlpapi:IPHLPAPI.DLL
 0003:00000128       __imp_IcmpSendEcho         000000018000c128     iphlpapi:IPHLPAPI.DLL
 0003:00000130       __imp_IcmpSendEcho2Ex      000000018000c130     iphlpapi:IPHLPAPI.DLL
 0003:00000138       __imp_GetAdaptersAddresses 000000018000c138     iphlpapi:IPHLPAPI.DLL
 0003:00000140       __imp_Icmp6SendEcho2       000000018000c140     iphlpapi:IPHLPAPI.DLL
 0003:00000148       __imp_GetIfEntry2          000000018000c148     iphlpapi:IPHLPAPI.DLL
 0003:00000150       __imp_GetIfTable2          000000018000c150     iphlpapi:IPHLPAPI.DLL
 0003:00000158       __imp_GetUnicastIpAddressTable 000000018000c158     iphlpapi:IPHLPAPI.DLL
 0003:00000160       \177IPHLPAPI_NULL_THUNK_DATA_DLA 000000018000c160     iphlpapi:IPHLPAPI.DLL
 0003:00000168       __imp_CompleteAuthToken    000000018000c168     secur32:Secur32.dll
 0003:00000170       __imp_InitializeSecurityContextA 000000018000c170     secur32:Secur32.dll
 0003:00000178       __imp_FreeCredentialsHandle 000000018000c178     secur32:Secur32.dll
 0003:00000180       __imp_AcquireCredentialsHandleA 000000018000c180     secur32:Secur32.dll
 0003:00000188       __imp_DeleteSecurityContext 000000018000c188     secur32:Secur32.dll
 0003:00000190       \177Secur32_NULL_THUNK_DATA_DLA 000000018000c190     secur32:Secur32.dll
 0003:000001f8       __hmod__Secur32_dll        000000018000c1f8     secur32:Secur32.dll
 0003:00000200       __hmod__IPHLPAPI_DLL       000000018000c200     iphlpapi:IPHLPAPI.DLL
 0003:00000208       ?DloadKernel32@@3PEAUHINSTANCE__@@EA 000000018000c208     delayimp:delayhlp.obj
 0003:00000210       ?DloadAcquireSRWLockExclusive@@3P6AXPEA_K@ZEA 000000018000c210     delayimp:delayhlp.obj
 0003:00000218       ?DloadReleaseSRWLockExclusive@@3P6AXPEA_K@ZEA 000000018000c218     delayimp:delayhlp.obj
 0003:00000220       ?DloadSrwLock@@3_KA        000000018000c220     delayimp:delayhlp.obj
 0003:00000228       ?DloadSectionLockCount@@3KA 000000018000c228     delayimp:delayhlp.obj
 0003:0000022c       ?DloadSectionOldProtection@@3KA 000000018000c22c     delayimp:delayhlp.obj
 0003:00000230       ?DloadSectionCommitPermanent@@3KA 000000018000c230     delayimp:delayhlp.obj
 0003:000007b0       ?__type_info_root_node@@3U__type_info_node@@A 000000018000c7b0     MSVCRT:tncleanup.obj
 0003:000007c0       __scrt_current_native_startup_state 000000018000c7c0     MSVCRT:utility.obj
 0003:000007c8       __scrt_native_startup_lock 000000018000c7c8     MSVCRT:utility.obj
 0003:00000808       __scrt_debugger_hook_flag  000000018000c808     MSVCRT:utility_desktop.obj
 0003:0000080c       __favor                    000000018000c80c     MSVCRT:cpu_disp.obj
 0003:00000810       ptype_socksID              000000018000c810     <common>
 0003:00000818       ptype_httpID               000000018000c818     <common>
 0003:00000820       pr_no_proxyID              000000018000c820     <common>
 0003:00000828       proxy_ctrID                000000018000c828     <common>
 0003:00000830       isaddr_createUnresolvedID  000000018000c830     <common>
 0003:00000838       ptype_class                000000018000c838     <common>
 0003:00000840       isaddr_class               000000018000c840     <common>
 0003:00000848       proxy_class                000000018000c848     <common>
 0003:00000850       ni_ibmaskID                000000018000c850     <common>
 0003:00000858       ni_ibbroadcastID           000000018000c858     <common>
 0003:00000860       ni_ibaddressID             000000018000c860     <common>
 0003:00000868       ni_ibctrID                 000000018000c868     <common>
 0003:00000870       ni_ibcls                   000000018000c870     <common>
 0003:00000878       ni_childsID                000000018000c878     <common>
 0003:00000880       ni_displayNameID           000000018000c880     <common>
 0003:00000888       ni_bindsID                 000000018000c888     <common>
 0003:00000890       ni_ctor                    000000018000c890     <common>
 0003:00000898       ni_addrsID                 000000018000c898     <common>
 0003:000008a0       ni_indexID                 000000018000c8a0     <common>
 0003:000008a8       ni_nameID                  000000018000c8a8     <common>
 0003:000008b0       ni_class                   000000018000c8b0     <common>
 0003:000008b8       ia_holderID                000000018000c8b8     <common>
 0003:000008c0       iac_class                  000000018000c8c0     <common>
 0003:000008c8       iac_origHostNameID         000000018000c8c8     <common>
 0003:000008d0       iac_hostNameID             000000018000c8d0     <common>
 0003:000008d8       iac_familyID               000000018000c8d8     <common>
 0003:000008e0       iac_addressID              000000018000c8e0     <common>
 0003:000008e8       ia_class                   000000018000c8e8     <common>
 0003:000008f0       ia6_ctrID                  000000018000c8f0     <common>
 0003:000008f8       ia6_scopeifnameID          000000018000c8f8     <common>
 0003:00000900       ia6_scopeidsetID           000000018000c900     <common>
 0003:00000908       ia6_scopeidID              000000018000c908     <common>
 0003:00000910       ia6_ipaddressID            000000018000c910     <common>
 0003:00000918       ia6_holder6ID              000000018000c918     <common>
 0003:00000920       ia6_class                  000000018000c920     <common>
 0003:00000928       ia4_ctrID                  000000018000c928     <common>
 0003:00000930       ia4_class                  000000018000c930     <common>
 0003:00000938       ?_OptionsStorage@?1??__local_stdio_scanf_options@@9@9 000000018000c938     <common>
 0003:00000940       ?_OptionsStorage@?1??__local_stdio_printf_options@@9@9 000000018000c940     <common>
 0003:00000948       __dyn_tls_init_callback    000000018000c948     <common>

 entry point at        0001:00006160

 Static symbols

 0000:ffff0000       .debug$S                   0000000180000000     net.exp
 0000:ffff0000       .debug$S                   0000000180000000     vcruntime:VCRUNTIME140.dll
 0000:ffff0000       .debug$S                   0000000180000000     vcruntime:VCRUNTIME140.dll
 0000:ffff0000       .debug$S                   0000000180000000     vcruntime:VCRUNTIME140.dll
 0000:ffff0000       .debug$S                   0000000180000000     vcruntime:VCRUNTIME140.dll
 0000:ffff0000       .debug$S                   0000000180000000     vcruntime:VCRUNTIME140.dll
 0000:ffff0000       .debug$S                   0000000180000000     vcruntime:VCRUNTIME140.dll
 0000:ffff0000       .debug$S                   0000000180000000     vcruntime:VCRUNTIME140.dll
 0000:ffff0000       .debug$S                   0000000180000000     vcruntime:VCRUNTIME140.dll
 0000:ffff0000       .debug$S                   0000000180000000     ucrt:api-ms-win-crt-heap-l1-1-0.dll
 0000:ffff0000       .debug$S                   0000000180000000     ucrt:api-ms-win-crt-heap-l1-1-0.dll
 0000:ffff0000       .debug$S                   0000000180000000     ucrt:api-ms-win-crt-heap-l1-1-0.dll
 0000:ffff0000       .debug$S                   0000000180000000     ucrt:api-ms-win-crt-runtime-l1-1-0.dll
 0000:ffff0000       .debug$S                   0000000180000000     ucrt:api-ms-win-crt-runtime-l1-1-0.dll
 0000:ffff0000       .debug$S                   0000000180000000     ucrt:api-ms-win-crt-runtime-l1-1-0.dll
 0000:ffff0000       .debug$S                   0000000180000000     ucrt:api-ms-win-crt-runtime-l1-1-0.dll
 0000:ffff0000       .debug$S                   0000000180000000     ucrt:api-ms-win-crt-runtime-l1-1-0.dll
 0000:ffff0000       .debug$S                   0000000180000000     ucrt:api-ms-win-crt-runtime-l1-1-0.dll
 0000:ffff0000       .debug$S                   0000000180000000     ucrt:api-ms-win-crt-runtime-l1-1-0.dll
 0000:ffff0000       .debug$S                   0000000180000000     ucrt:api-ms-win-crt-runtime-l1-1-0.dll
 0000:ffff0000       .debug$S                   0000000180000000     ucrt:api-ms-win-crt-runtime-l1-1-0.dll
 0000:ffff0000       .debug$S                   0000000180000000     ucrt:api-ms-win-crt-runtime-l1-1-0.dll
 0000:ffff0000       .debug$S                   0000000180000000     ucrt:api-ms-win-crt-runtime-l1-1-0.dll
 0000:ffff0000       .debug$S                   0000000180000000     ucrt:api-ms-win-crt-runtime-l1-1-0.dll
 0000:ffff0000       .debug$S                   0000000180000000     ucrt:api-ms-win-crt-runtime-l1-1-0.dll
 0000:ffff0000       .debug$S                   0000000180000000     ucrt:api-ms-win-crt-stdio-l1-1-0.dll
 0000:ffff0000       .debug$S                   0000000180000000     ucrt:api-ms-win-crt-stdio-l1-1-0.dll
 0000:ffff0000       .debug$S                   0000000180000000     ucrt:api-ms-win-crt-stdio-l1-1-0.dll
 0000:ffff0000       .debug$S                   0000000180000000     ucrt:api-ms-win-crt-stdio-l1-1-0.dll
 0000:ffff0000       .debug$S                   0000000180000000     ucrt:api-ms-win-crt-stdio-l1-1-0.dll
 0000:ffff0000       .debug$S                   0000000180000000     ucrt:api-ms-win-crt-string-l1-1-0.dll
 0000:ffff0000       .debug$S                   0000000180000000     ucrt:api-ms-win-crt-string-l1-1-0.dll
 0000:ffff0000       .debug$S                   0000000180000000     ucrt:api-ms-win-crt-string-l1-1-0.dll
 0000:ffff0000       .debug$S                   0000000180000000     ucrt:api-ms-win-crt-string-l1-1-0.dll
 0000:ffff0000       .debug$S                   0000000180000000     ucrt:api-ms-win-crt-string-l1-1-0.dll
 0000:ffff0000       .debug$S                   0000000180000000     ucrt:api-ms-win-crt-string-l1-1-0.dll
 0000:ffff0000       .debug$S                   0000000180000000     ucrt:api-ms-win-crt-string-l1-1-0.dll
 0000:ffff0000       .debug$S                   0000000180000000     ucrt:api-ms-win-crt-string-l1-1-0.dll
 0000:ffff0000       .debug$S                   0000000180000000     advapi32:ADVAPI32.dll
 0000:ffff0000       .debug$S                   0000000180000000     advapi32:ADVAPI32.dll
 0000:ffff0000       .debug$S                   0000000180000000     advapi32:ADVAPI32.dll
 0000:ffff0000       .debug$S                   0000000180000000     iphlpapi:IPHLPAPI.DLL
 0000:ffff0000       .debug$S                   0000000180000000     iphlpapi:IPHLPAPI.DLL
 0000:ffff0000       .debug$S                   0000000180000000     iphlpapi:IPHLPAPI.DLL
 0000:ffff0000       .debug$S                   0000000180000000     iphlpapi:IPHLPAPI.DLL
 0000:ffff0000       .debug$S                   0000000180000000     iphlpapi:IPHLPAPI.DLL
 0000:ffff0000       .debug$S                   0000000180000000     iphlpapi:IPHLPAPI.DLL
 0000:ffff0000       .debug$S                   0000000180000000     iphlpapi:IPHLPAPI.DLL
 0000:ffff0000       .debug$S                   0000000180000000     iphlpapi:IPHLPAPI.DLL
 0000:ffff0000       .debug$S                   0000000180000000     iphlpapi:IPHLPAPI.DLL
 0000:ffff0000       .debug$S                   0000000180000000     iphlpapi:IPHLPAPI.DLL
 0000:ffff0000       .debug$S                   0000000180000000     iphlpapi:IPHLPAPI.DLL
 0000:ffff0000       .debug$S                   0000000180000000     iphlpapi:IPHLPAPI.DLL
 0000:ffff0000       .debug$S                   0000000180000000     iphlpapi:IPHLPAPI.DLL
 0000:ffff0000       .debug$S                   0000000180000000     iphlpapi:IPHLPAPI.DLL
 0000:ffff0000       .debug$S                   0000000180000000     iphlpapi:IPHLPAPI.DLL
 0000:ffff0000       .debug$S                   0000000180000000     iphlpapi:IPHLPAPI.DLL
 0000:ffff0000       .debug$S                   0000000180000000     kernel32:KERNEL32.dll
 0000:ffff0000       .debug$S                   0000000180000000     kernel32:KERNEL32.dll
 0000:ffff0000       .debug$S                   0000000180000000     kernel32:KERNEL32.dll
 0000:ffff0000       .debug$S                   0000000180000000     kernel32:KERNEL32.dll
 0000:ffff0000       .debug$S                   0000000180000000     kernel32:KERNEL32.dll
 0000:ffff0000       .debug$S                   0000000180000000     kernel32:KERNEL32.dll
 0000:ffff0000       .debug$S                   0000000180000000     kernel32:KERNEL32.dll
 0000:ffff0000       .debug$S                   0000000180000000     kernel32:KERNEL32.dll
 0000:ffff0000       .debug$S                   0000000180000000     kernel32:KERNEL32.dll
 0000:ffff0000       .debug$S                   0000000180000000     kernel32:KERNEL32.dll
 0000:ffff0000       .debug$S                   0000000180000000     kernel32:KERNEL32.dll
 0000:ffff0000       .debug$S                   0000000180000000     kernel32:KERNEL32.dll
 0000:ffff0000       .debug$S                   0000000180000000     kernel32:KERNEL32.dll
 0000:ffff0000       .debug$S                   0000000180000000     kernel32:KERNEL32.dll
 0000:ffff0000       .debug$S                   0000000180000000     kernel32:KERNEL32.dll
 0000:ffff0000       .debug$S                   0000000180000000     kernel32:KERNEL32.dll
 0000:ffff0000       .debug$S                   0000000180000000     kernel32:KERNEL32.dll
 0000:ffff0000       .debug$S                   0000000180000000     kernel32:KERNEL32.dll
 0000:ffff0000       .debug$S                   0000000180000000     kernel32:KERNEL32.dll
 0000:ffff0000       .debug$S                   0000000180000000     kernel32:KERNEL32.dll
 0000:ffff0000       .debug$S                   0000000180000000     kernel32:KERNEL32.dll
 0000:ffff0000       .debug$S                   0000000180000000     kernel32:KERNEL32.dll
 0000:ffff0000       .debug$S                   0000000180000000     kernel32:KERNEL32.dll
 0000:ffff0000       .debug$S                   0000000180000000     kernel32:KERNEL32.dll
 0000:ffff0000       .debug$S                   0000000180000000     kernel32:KERNEL32.dll
 0000:ffff0000       .debug$S                   0000000180000000     kernel32:KERNEL32.dll
 0000:ffff0000       .debug$S                   0000000180000000     kernel32:KERNEL32.dll
 0000:ffff0000       .debug$S                   0000000180000000     kernel32:KERNEL32.dll
 0000:ffff0000       .debug$S                   0000000180000000     kernel32:KERNEL32.dll
 0000:ffff0000       .debug$S                   0000000180000000     kernel32:KERNEL32.dll
 0000:ffff0000       .debug$S                   0000000180000000     kernel32:KERNEL32.dll
 0000:ffff0000       .debug$S                   0000000180000000     kernel32:KERNEL32.dll
 0000:ffff0000       .debug$S                   0000000180000000     kernel32:KERNEL32.dll
 0000:ffff0000       .debug$S                   0000000180000000     secur32:Secur32.dll
 0000:ffff0000       .debug$S                   0000000180000000     secur32:Secur32.dll
 0000:ffff0000       .debug$S                   0000000180000000     secur32:Secur32.dll
 0000:ffff0000       .debug$S                   0000000180000000     secur32:Secur32.dll
 0000:ffff0000       .debug$S                   0000000180000000     secur32:Secur32.dll
 0000:ffff0000       .debug$S                   0000000180000000     winhttp:WINHTTP.dll
 0000:ffff0000       .debug$S                   0000000180000000     winhttp:WINHTTP.dll
 0000:ffff0000       .debug$S                   0000000180000000     winhttp:WINHTTP.dll
 0000:ffff0000       .debug$S                   0000000180000000     ws2_32:WS2_32.dll
 0000:ffff0000       .debug$S                   0000000180000000     ws2_32:WS2_32.dll
 0000:ffff0000       .debug$S                   0000000180000000     ws2_32:WS2_32.dll
 0000:ffff0000       .debug$S                   0000000180000000     ws2_32:WS2_32.dll
 0000:ffff0000       .debug$S                   0000000180000000     ws2_32:WS2_32.dll
 0000:ffff0000       .debug$S                   0000000180000000     ws2_32:WS2_32.dll
 0000:ffff0000       .debug$S                   0000000180000000     ws2_32:WS2_32.dll
 0000:ffff0000       .debug$S                   0000000180000000     ws2_32:WS2_32.dll
 0000:ffff0000       .debug$S                   0000000180000000     ws2_32:WS2_32.dll
 0000:ffff0000       .debug$S                   0000000180000000     ws2_32:WS2_32.dll
 0000:ffff0000       .debug$S                   0000000180000000     ws2_32:WS2_32.dll
 0000:ffff0000       .debug$S                   0000000180000000     ws2_32:WS2_32.dll
 0000:ffff0000       .debug$S                   0000000180000000     ws2_32:WS2_32.dll
 0000:ffff0000       .debug$S                   0000000180000000     ws2_32:WS2_32.dll
 0000:ffff0000       .debug$S                   0000000180000000     ws2_32:WS2_32.dll
 0000:ffff0000       .debug$S                   0000000180000000     ws2_32:WS2_32.dll
 0000:ffff0000       .debug$S                   0000000180000000     ws2_32:WS2_32.dll
 0000:ffff0000       .debug$S                   0000000180000000     ws2_32:WS2_32.dll
 0000:ffff0000       .debug$S                   0000000180000000     ws2_32:WS2_32.dll
 0000:ffff0000       .debug$S                   0000000180000000     ws2_32:WS2_32.dll
 0000:ffff0000       .debug$S                   0000000180000000     ws2_32:WS2_32.dll
 0000:ffff0000       .debug$S                   0000000180000000     ws2_32:WS2_32.dll
 0000:ffff0000       .debug$S                   0000000180000000     ws2_32:WS2_32.dll
 0000:ffff0000       .debug$S                   0000000180000000     ws2_32:WS2_32.dll
 0000:ffff0000       .debug$S                   0000000180000000     ws2_32:WS2_32.dll
 0000:ffff0000       .debug$S                   0000000180000000     jvm:jvm.dll
 0000:ffff0000       .debug$S                   0000000180000000     jvm:jvm.dll
 0000:ffff0000       .debug$S                   0000000180000000     java:java.dll
 0000:ffff0000       .debug$S                   0000000180000000     java:java.dll
 0000:ffff0000       .debug$S                   0000000180000000     java:java.dll
 0000:ffff0000       .debug$S                   0000000180000000     java:java.dll
 0000:ffff0000       .debug$S                   0000000180000000     java:java.dll
 0000:ffff0000       .debug$S                   0000000180000000     java:java.dll
 0000:ffff0000       .debug$S                   0000000180000000     java:java.dll
 0000:ffff0000       .debug$S                   0000000180000000     java:java.dll
 0000:ffff0000       .debug$S                   0000000180000000     java:java.dll
 0001:000005a0       createProxyList            00000001800015a0 f   DefaultProxySelector.obj
 0001:00000da0       ping4                      0000000180001da0 f   Inet4AddressImpl.obj
 0001:00001004       tcp_ping4                  0000000180002004 f   Inet4AddressImpl.obj
 0001:00001ae8       ping6                      0000000180002ae8 f   Inet6AddressImpl.obj
 0001:00001c00       tcp_ping6                  0000000180002c00 f   Inet6AddressImpl.obj
 0001:0000247c       endSequence                000000018000347c f   NTLMAuthSequence.obj
 0001:000030c4       createNetworkInterface     00000001800040c4 f   NetworkInterface.obj
 0001:00003828       createNetworkInterfaceForSingleRow 0000000180004828 f   NetworkInterface.obj
 0001:0000388c       createNetworkInterfaceForSingleRowWithTables 000000018000488c f   NetworkInterface.obj
 0001:00003908       getAddressTables           0000000180004908 f   NetworkInterface.obj
 0001:00003b34       loadConfig                 0000000180004b34 f   ResolverConfigurationImpl.obj
 0001:00005e10       $$000000                   0000000180006e10     MSVCRT:amdsecgs.obj
 0001:00005e40       ?dllmain_crt_dispatch@@YAHQEAUHINSTANCE__@@KQEAX@Z 0000000180006e40 f   MSVCRT:dll_dllmain.obj
 0001:00005e90       ?dllmain_crt_process_attach@@YAHQEAUHINSTANCE__@@QEAX@Z 0000000180006e90 f   MSVCRT:dll_dllmain.obj
 0001:00005fa8       ?dllmain_crt_process_detach@@YAH_N@Z 0000000180006fa8 f   MSVCRT:dll_dllmain.obj
 0001:0000602c       ?dllmain_dispatch@@YAHQEAUHINSTANCE__@@KQEAX@Z 000000018000702c f   MSVCRT:dll_dllmain.obj
 0001:000062ac       capture_previous_context   00000001800072ac f   MSVCRT:gs_report.obj
 0001:00006b40       $$000000                   0000000180007b40     MSVCRT:guard_dispatch.obj
 0001:00006b60       $$000000                   0000000180007b60     MSVCRT:guard_xfg_dispatch.obj
 0001:00006b76       ?fin$0@?0??dllmain_crt_process_attach@@YAHQEAUHINSTANCE__@@QEAX@Z@4HA 0000000180007b76 f   MSVCRT:dll_dllmain.obj
 0001:00006b8d       ?fin$0@?0??dllmain_crt_process_detach@@YAH_N@Z@4HA 0000000180007b8d f   MSVCRT:dll_dllmain.obj
 0001:00006ba6       ?fin$1@?0??dllmain_crt_process_detach@@YAH_N@Z@4HA 0000000180007ba6 f   MSVCRT:dll_dllmain.obj
 0001:00006bba       ?filt$0@?0??dllmain_dispatch@@YAHQEAUHINSTANCE__@@KQEAX@Z@4HA 0000000180007bba f   MSVCRT:dll_dllmain.obj
 0001:00006bf0       __scrt_is_nonwritable_in_current_image$filt$0 0000000180007bf0 f   MSVCRT:utility.obj
 0002:00000410       ?separators@?1??createProxyList@@9@9 0000000180008410     DefaultProxySelector.obj
 0002:00000c50       winsock_errors             0000000180008c50     net_util_md.obj
 0002:00001a00       GS_ExceptionPointers       0000000180009a00     MSVCRT:gs_report.obj
 0002:00001ee0       $unwind$swprintf           0000000180009ee0     DefaultProxySelector.obj
 0002:00001ee0       $unwind$snprintf           0000000180009ee0     net_util_md.obj
 0002:00001ef0       $unwind$swscanf            0000000180009ef0     DefaultProxySelector.obj
 0002:00001efc       $unwind$Java_sun_net_spi_DefaultProxySelector_init 0000000180009efc     DefaultProxySelector.obj
 0002:00001f04       $unwind$Java_sun_net_spi_DefaultProxySelector_getSystemProxies 0000000180009f04     DefaultProxySelector.obj
 0002:00001f28       $unwind$createProxyList    0000000180009f28     DefaultProxySelector.obj
 0002:00001f40       $unwind$Java_java_net_Inet4Address_init 0000000180009f40     Inet4Address.obj
 0002:00001f40       $unwind$Java_java_net_InetAddress_init 0000000180009f40     InetAddress.obj
 0002:00001f40       $unwind$Java_java_net_NetworkInterface_init 0000000180009f40     NetworkInterface.obj
 0002:00001f40       $unwind$initInetAddressIDs 0000000180009f40     net_util.obj
 0002:00001f40       $unwind$NET_Bind           0000000180009f40     net_util_md.obj
 0002:00001f40       $unwind$NET_Socket         0000000180009f40     net_util_md.obj
 0002:00001f40       $unwind$NET_SocketAvailable 0000000180009f40     net_util_md.obj
 0002:00001f40       $unwind$__raise_securityfailure 0000000180009f40     MSVCRT:gs_report.obj
 0002:00001f40       $unwind$__scrt_initialize_crt 0000000180009f40     MSVCRT:utility.obj
 0002:00001f40       $unwind$__scrt_initialize_onexit_tables 0000000180009f40     MSVCRT:utility.obj
 0002:00001f40       $unwind$__scrt_release_startup_lock 0000000180009f40     MSVCRT:utility.obj
 0002:00001f40       $unwind$__scrt_uninitialize_crt 0000000180009f40     MSVCRT:utility.obj
 0002:00001f40       $unwind$?DloadAcquireSectionWriteAccess@@YAXXZ 0000000180009f40     delayimp:delayhlp.obj
 0002:00001f48       $unwind$Java_java_net_Inet4AddressImpl_getLocalHostName 0000000180009f48     Inet4AddressImpl.obj
 0002:00001f48       $unwind$Java_java_net_Inet6AddressImpl_getLocalHostName 0000000180009f48     Inet6AddressImpl.obj
 0002:00001f5c       $unwind$Java_java_net_Inet4AddressImpl_lookupAllHostAddr 0000000180009f5c     Inet4AddressImpl.obj
 0002:00001f78       $unwind$Java_java_net_Inet4AddressImpl_getHostByAddr 0000000180009f78     Inet4AddressImpl.obj
 0002:00001f94       $unwind$Java_java_net_Inet4AddressImpl_isReachable0 0000000180009f94     Inet4AddressImpl.obj
 0002:00001fb0       $unwind$tcp_ping4          0000000180009fb0     Inet4AddressImpl.obj
 0002:00001fb0       $unwind$tcp_ping6          0000000180009fb0     Inet6AddressImpl.obj
 0002:00001fcc       $unwind$ping4              0000000180009fcc     Inet4AddressImpl.obj
 0002:00001fe8       $unwind$Java_java_net_Inet6Address_init 0000000180009fe8     Inet6Address.obj
 0002:00001fe8       $unwind$createNetworkInterfaceForSingleRow 0000000180009fe8     NetworkInterface.obj
 0002:00001fe8       $unwind$Java_sun_net_dns_ResolverConfigurationImpl_init0 0000000180009fe8     ResolverConfigurationImpl.obj
 0002:00001fe8       $unwind$initJavaClass      0000000180009fe8     proxy_util.obj
 0002:00001fe8       $unwind$_RTC_Initialize    0000000180009fe8     MSVCRT:initsect.obj
 0002:00001fe8       $unwind$_RTC_Terminate     0000000180009fe8     MSVCRT:initsect.obj
 0002:00001fe8       $unwind$?DloadGetSRWLockFunctionPointers@@YAEXZ 0000000180009fe8     delayimp:delayhlp.obj
 0002:00001ff4       $unwind$Java_java_net_Inet6AddressImpl_lookupAllHostAddr 0000000180009ff4     Inet6AddressImpl.obj
 0002:0000200c       $unwind$Java_java_net_Inet6AddressImpl_getHostByAddr 000000018000a00c     Inet6AddressImpl.obj
 0002:0000202c       $unwind$Java_java_net_Inet6AddressImpl_isReachable0 000000018000a02c     Inet6AddressImpl.obj
 0002:0000204c       $unwind$ping6              000000018000a04c     Inet6AddressImpl.obj
 0002:0000206c       $unwind$endSequence        000000018000a06c     NTLMAuthSequence.obj
 0002:0000206c       $unwind$createNetworkInterfaceForSingleRowWithTables 000000018000a06c     NetworkInterface.obj
 0002:0000206c       $unwind$getAddressTables   000000018000a06c     NetworkInterface.obj
 0002:0000206c       $unwind$strappend          000000018000a06c     ResolverConfigurationImpl.obj
 0002:0000206c       $unwind$__scrt_dllmain_exception_filter 000000018000a06c     MSVCRT:utility.obj
 0002:00002080       $unwind$Java_sun_net_www_protocol_http_ntlm_NTLMAuthSequence_initFirst 000000018000a080     NTLMAuthSequence.obj
 0002:00002080       $unwind$getInet6Address_scopeid 000000018000a080     net_util.obj
 0002:00002080       $unwind$getInetAddress_addr 000000018000a080     net_util.obj
 0002:00002080       $unwind$getInetAddress_family 000000018000a080     net_util.obj
 0002:00002080       $unwind$setInet6Address_scopeid 000000018000a080     net_util.obj
 0002:00002080       $unwind$setInet6Address_scopeifname 000000018000a080     net_util.obj
 0002:00002080       $unwind$setInetAddress_addr 000000018000a080     net_util.obj
 0002:00002080       $unwind$setInetAddress_family 000000018000a080     net_util.obj
 0002:00002080       $unwind$setInetAddress_hostName 000000018000a080     net_util.obj
 0002:00002080       $unwind$NET_WinBind        000000018000a080     net_util_md.obj
 0002:00002080       $unwind$_DllMainCRTStartup 000000018000a080     MSVCRT:dll_dllmain.obj
 0002:00002090       $unwind$Java_sun_net_www_protocol_http_ntlm_NTLMAuthSequence_getCredentialsHandle 000000018000a090     NTLMAuthSequence.obj
 0002:000020ac       $unwind$Java_sun_net_www_protocol_http_ntlm_NTLMAuthSequence_getNextToken 000000018000a0ac     NTLMAuthSequence.obj
 0002:000020cc       $unwind$Java_sun_net_www_protocol_http_ntlm_NTLMAuthentication_isTrustedSiteAvailable 000000018000a0cc     NTLMAuthentication.obj
 0002:000020cc       $unwind$NET_GetPortFromSockaddr 000000018000a0cc     net_util.obj
 0002:000020cc       $unwind$IPv4_supported     000000018000a0cc     net_util_md.obj
 0002:000020cc       $unwind$IPv6_supported     000000018000a0cc     net_util_md.obj
 0002:000020cc       $unwind$__scrt_initialize_default_local_stdio_options 000000018000a0cc     MSVCRT:default_local_stdio_options.obj
 0002:000020cc       $unwind$?dllmain_crt_dispatch@@YAHQEAUHINSTANCE__@@KQEAX@Z 000000018000a0cc     MSVCRT:dll_dllmain.obj
 0002:000020cc       $unwind$__GSHandlerCheck   000000018000a0cc     MSVCRT:gshandler.obj
 0002:000020cc       $unwind$__scrt_acquire_startup_lock 000000018000a0cc     MSVCRT:utility.obj
 0002:000020cc       $unwind$__scrt_dllmain_after_initialize_c 000000018000a0cc     MSVCRT:utility.obj
 0002:000020cc       $unwind$__scrt_dllmain_before_initialize_c 000000018000a0cc     MSVCRT:utility.obj
 0002:000020cc       $unwind$__scrt_dllmain_crt_thread_attach 000000018000a0cc     MSVCRT:utility.obj
 0002:000020cc       $unwind$__scrt_dllmain_crt_thread_detach 000000018000a0cc     MSVCRT:utility.obj
 0002:000020cc       $unwind$__scrt_dllmain_uninitialize_c 000000018000a0cc     MSVCRT:utility.obj
 0002:000020cc       $unwind$__scrt_dllmain_uninitialize_critical 000000018000a0cc     MSVCRT:utility.obj
 0002:000020cc       $unwind$?DloadReleaseSectionWriteAccess@@YAXXZ 000000018000a0cc     delayimp:delayhlp.obj
 0002:000020d4       $unwind$Java_sun_net_www_protocol_http_ntlm_NTLMAuthentication_isTrustedSite0 000000018000a0d4     NTLMAuthentication.obj
 0002:000020e8       $unwind$Java_java_net_NetworkInterface_getAll 000000018000a0e8     NetworkInterface.obj
 0002:000020fc       $unwind$Java_java_net_NetworkInterface_getByName0 000000018000a0fc     NetworkInterface.obj
 0002:00002118       $unwind$Java_java_net_NetworkInterface_getByIndex0 000000018000a118     NetworkInterface.obj
 0002:00002118       $unwind$Java_java_net_NetworkInterface_getMTU0 000000018000a118     NetworkInterface.obj
 0002:00002118       $unwind$Java_java_net_NetworkInterface_isLoopback0 000000018000a118     NetworkInterface.obj
 0002:00002118       $unwind$Java_java_net_NetworkInterface_isP2P0 000000018000a118     NetworkInterface.obj
 0002:00002118       $unwind$Java_java_net_NetworkInterface_isUp0 000000018000a118     NetworkInterface.obj
 0002:00002130       $unwind$Java_java_net_NetworkInterface_boundInetAddress0 000000018000a130     NetworkInterface.obj
 0002:00002144       $unwind$Java_java_net_NetworkInterface_getByInetAddress0 000000018000a144     NetworkInterface.obj
 0002:00002164       $unwind$Java_java_net_NetworkInterface_getMacAddr0 000000018000a164     NetworkInterface.obj
 0002:0000217c       $unwind$createNetworkInterface 000000018000a17c     NetworkInterface.obj
 0002:000021a0       $unwind$loadConfig         000000018000a1a0     ResolverConfigurationImpl.obj
 0002:000021c0       $unwind$Java_sun_net_dns_ResolverConfigurationImpl_loadDNSconfig0 000000018000a1c0     ResolverConfigurationImpl.obj
 0002:000021d8       $unwind$Java_sun_net_dns_ResolverConfigurationImpl_notifyAddrChange0 000000018000a1d8     ResolverConfigurationImpl.obj
 0002:000021e0       $unwind$JNI_OnLoad         000000018000a1e0     net_util.obj
 0002:000021f0       $unwind$getInet6Address_ipaddress 000000018000a1f0     net_util.obj
 0002:000021f0       $unwind$setInet6Address_ipaddress 000000018000a1f0     net_util.obj
 0002:000021f0       $unwind$NET_GetSockOpt     000000018000a1f0     net_util_md.obj
 0002:00002204       $unwind$NET_SockaddrToInetAddress 000000018000a204     net_util.obj
 0002:0000221c       $unwind$NET_SockaddrEqualsInetAddress 000000018000a21c     net_util.obj
 0002:00002234       $unwind$NET_EnableFastTcpLoopbackConnect 000000018000a234     net_util_md.obj
 0002:00002240       $unwind$NET_ThrowNew       000000018000a240     net_util_md.obj
 0002:00002258       $unwind$NET_InetAddressToSockaddr 000000018000a258     net_util_md.obj
 0002:00002274       $unwind$NET_SetSockOpt     000000018000a274     net_util_md.obj
 0002:00002288       $unwind$NET_EnableFastTcpLoopback 000000018000a288     net_util_md.obj
 0002:00002290       $unwind$NET_Wait           000000018000a290     net_util_md.obj
 0002:000022b4       $unwind$DllMain            000000018000a2b4     net_util_md.obj
 0002:000022c4       $unwind$setExclusiveBind   000000018000a2c4     net_util_md.obj
 0002:000022cc       $unwind$IsWindows10RS3OrGreater 000000018000a2cc     net_util_md.obj
 0002:000022e0       xdata                      000000018000a2e0     secur32:Secur32.dll
 0002:000022e8       xdata                      000000018000a2e8     iphlpapi:IPHLPAPI.DLL
 0002:000022f0       $unwind$?DloadObtainSection@@YAPEAXPEAK0@Z 000000018000a2f0     delayimp:delayhlp.obj
 0002:00002300       $unwind$?DloadMakePermanentImageCommit@@YAXPEAX_K@Z 000000018000a300     delayimp:delayhlp.obj
 0002:0000230c       $unwind$?DloadProtectSection@@YAXKPEAK@Z 000000018000a30c     delayimp:delayhlp.obj
 0002:0000231c       $unwind$__delayLoadHelper2 000000018000a31c     delayimp:delayhlp.obj
 0002:00002338       $unwind$__GSHandlerCheckCommon 000000018000a338     MSVCRT:gshandler.obj
 0002:00002340       $xdatasym                  000000018000a340     MSVCRT:amdsecgs.obj
 0002:00002344       $unwind$?dllmain_crt_process_attach@@YAHQEAUHINSTANCE__@@QEAX@Z 000000018000a344     MSVCRT:dll_dllmain.obj
 0002:00002380       $unwind$?fin$0@?0??dllmain_crt_process_attach@@YAHQEAUHINSTANCE__@@QEAX@Z@4HA 000000018000a380     MSVCRT:dll_dllmain.obj
 0002:00002380       $unwind$?fin$0@?0??dllmain_crt_process_detach@@YAH_N@Z@4HA 000000018000a380     MSVCRT:dll_dllmain.obj
 0002:00002380       $unwind$?fin$1@?0??dllmain_crt_process_detach@@YAH_N@Z@4HA 000000018000a380     MSVCRT:dll_dllmain.obj
 0002:00002388       $unwind$?dllmain_crt_process_detach@@YAH_N@Z 000000018000a388     MSVCRT:dll_dllmain.obj
 0002:000023dc       $unwind$?dllmain_dispatch@@YAHQEAUHINSTANCE__@@KQEAX@Z 000000018000a3dc     MSVCRT:dll_dllmain.obj
 0002:00002404       $unwind$?filt$0@?0??dllmain_dispatch@@YAHQEAUHINSTANCE__@@KQEAX@Z@4HA 000000018000a404     MSVCRT:dll_dllmain.obj
 0002:0000240c       $unwind$__report_gsfailure 000000018000a40c     MSVCRT:gs_report.obj
 0002:00002414       $unwind$capture_previous_context 000000018000a414     MSVCRT:gs_report.obj
 0002:00002420       $unwind$__security_init_cookie 000000018000a420     MSVCRT:gs_support.obj
 0002:0000242c       $unwind$__scrt_is_nonwritable_in_current_image 000000018000a42c     MSVCRT:utility.obj
 0002:0000244c       $unwind$__scrt_is_nonwritable_in_current_image$filt$0 000000018000a44c     MSVCRT:utility.obj
 0002:00002454       $unwind$__scrt_fastfail    000000018000a454     MSVCRT:utility_desktop.obj
 0002:00002468       $xdatasym                  000000018000a468     MSVCRT:guard_dispatch.obj
 0002:00002470       $xdatasym                  000000018000a470     MSVCRT:guard_xfg_dispatch.obj
 0002:00002474       $unwind$__isa_available_init 000000018000a474     MSVCRT:cpu_disp.obj
 0002:00002830       .edata                     000000018000a830     net.exp
 0002:00002858       rgpv                       000000018000a858     net.exp
 0002:00002930       rgszName                   000000018000a930     net.exp
 0002:00002a08       rgwOrd                     000000018000aa08     net.exp
 0002:00002a74       szName                     000000018000aa74     net.exp
 0002:00002a7c       $N00001                    000000018000aa7c     net.exp
 0002:00002a87       $N00002                    000000018000aa87     net.exp
 0002:00002ab4       $N00003                    000000018000aab4     net.exp
 0002:00002ae4       $N00004                    000000018000aae4     net.exp
 0002:00002b10       $N00005                    000000018000ab10     net.exp
 0002:00002b41       $N00006                    000000018000ab41     net.exp
 0002:00002b61       $N00007                    000000018000ab61     net.exp
 0002:00002b8e       $N00008                    000000018000ab8e     net.exp
 0002:00002bbe       $N00009                    000000018000abbe     net.exp
 0002:00002bea       $N00010                    000000018000abea     net.exp
 0002:00002c1b       $N00011                    000000018000ac1b     net.exp
 0002:00002c3b       $N00012                    000000018000ac3b     net.exp
 0002:00002c5a       $N00013                    000000018000ac5a     net.exp
 0002:00002c84       $N00014                    000000018000ac84     net.exp
 0002:00002cae       $N00015                    000000018000acae     net.exp
 0002:00002cdf       $N00016                    000000018000acdf     net.exp
 0002:00002d05       $N00017                    000000018000ad05     net.exp
 0002:00002d30       $N00018                    000000018000ad30     net.exp
 0002:00002d61       $N00019                    000000018000ad61     net.exp
 0002:00002d8b       $N00020                    000000018000ad8b     net.exp
 0002:00002db2       $N00021                    000000018000adb2     net.exp
 0002:00002ddd       $N00022                    000000018000addd     net.exp
 0002:00002e01       $N00023                    000000018000ae01     net.exp
 0002:00002e2c       $N00024                    000000018000ae2c     net.exp
 0002:00002e52       $N00025                    000000018000ae52     net.exp
 0002:00002e77       $N00026                    000000018000ae77     net.exp
 0002:00002ea9       $N00027                    000000018000aea9     net.exp
 0002:00002eda       $N00028                    000000018000aeda     net.exp
 0002:00002f14       $N00029                    000000018000af14     net.exp
 0002:00002f51       $N00030                    000000018000af51     net.exp
 0002:00002f88       $N00031                    000000018000af88     net.exp
 0002:00002fb3       $N00032                    000000018000afb3     net.exp
 0002:00002ffd       $N00033                    000000018000affd     net.exp
 0002:0000303f       $N00034                    000000018000b03f     net.exp
 0002:0000307e       $N00035                    000000018000b07e     net.exp
 0002:000030c4       $N00036                    000000018000b0c4     net.exp
 0002:00003112       $N00037                    000000018000b112     net.exp
 0002:0000311b       $N00038                    000000018000b11b     net.exp
 0002:00003135       $N00039                    000000018000b135     net.exp
 0002:00003156       $N00040                    000000018000b156     net.exp
 0002:0000316e       $N00041                    000000018000b16e     net.exp
 0002:0000317d       $N00042                    000000018000b17d     net.exp
 0002:00003197       $N00043                    000000018000b197     net.exp
 0002:000031ab       $N00044                    000000018000b1ab     net.exp
 0002:000031c1       $N00045                    000000018000b1c1     net.exp
 0002:000031d0       $N00046                    000000018000b1d0     net.exp
 0002:000031ee       $N00047                    000000018000b1ee     net.exp
 0002:00003208       $N00048                    000000018000b208     net.exp
 0002:0000321c       $N00049                    000000018000b21c     net.exp
 0002:00003229       $N00050                    000000018000b229     net.exp
 0002:00003235       $N00051                    000000018000b235     net.exp
 0002:00003248       $N00052                    000000018000b248     net.exp
 0002:00003257       $N00053                    000000018000b257     net.exp
 0002:00003266       $N00054                    000000018000b266     net.exp
 0002:00003782       .idata$6                   000000018000b782     ws2_32:WS2_32.dll
 0002:000037b6       .idata$6                   000000018000b7b6     jvm:jvm.dll
 0002:0000380c       .idata$6                   000000018000b80c     winhttp:WINHTTP.dll
 0002:00003920       .idata$6                   000000018000b920     java:java.dll
 0002:0000395c       .idata$6                   000000018000b95c     advapi32:ADVAPI32.dll
 0002:00003bfa       .idata$6                   000000018000bbfa     kernel32:KERNEL32.dll
 0002:00003c68       .idata$6                   000000018000bc68     vcruntime:VCRUNTIME140.dll
 0002:00003de8       .idata$6                   000000018000bde8     ucrt:api-ms-win-crt-string-l1-1-0.dll
 0002:00003e0a       .idata$6                   000000018000be0a     ucrt:api-ms-win-crt-stdio-l1-1-0.dll
 0002:00003e2a       .idata$6                   000000018000be2a     ucrt:api-ms-win-crt-heap-l1-1-0.dll
 0002:00003e4a       .idata$6                   000000018000be4a     ucrt:api-ms-win-crt-runtime-l1-1-0.dll
 0003:00000010       ?opts@?1??NET_MapSocketOption@@9@9 000000018000c010     net_util_md.obj
 0003:000001a0       session                    000000018000c1a0     DefaultProxySelector.obj
 0003:000001a8       ia4_initialized            000000018000c1a8     Inet4Address.obj
 0003:000001ac       ia6_initialized            000000018000c1ac     Inet6Address.obj
 0003:000001b0       ia_initialized             000000018000c1b0     InetAddress.obj
 0003:000001b8       ntlm_ctxHandleID           000000018000c1b8     NTLMAuthSequence.obj
 0003:000001c0       ntlm_crdHandleID           000000018000c1c0     NTLMAuthSequence.obj
 0003:000001c8       status_seqCompleteID       000000018000c1c8     NTLMAuthSequence.obj
 0003:000001d0       fn_CoInternetCreateSecurityManager 000000018000c1d0     NTLMAuthentication.obj
 0003:000001d8       searchlistID               000000018000c1d8     ResolverConfigurationImpl.obj
 0003:000001e0       nameserversID              000000018000c1e0     ResolverConfigurationImpl.obj
 0003:000001e8       IPv4_available             000000018000c1e8     net_util.obj
 0003:000001ec       IPv6_available             000000018000c1ec     net_util.obj
 0003:000001f0       REUSEPORT_available        000000018000c1f0     net_util.obj
 0003:000001f4       initialized                000000018000c1f4     net_util.obj
 0003:00000234       ?__proc_attached@@3HA      000000018000c234     MSVCRT:dll_dllmain.obj
 0003:00000240       GS_ExceptionRecord         000000018000c240     MSVCRT:gs_report.obj
 0003:000002e0       GS_ContextRecord           000000018000c2e0     MSVCRT:gs_report.obj
 0003:000007d0       ?is_initialized_as_dll@@3_NA 000000018000c7d0     MSVCRT:utility.obj
 0003:000007d1       ?module_local_atexit_table_initialized@@3_NA 000000018000c7d1     MSVCRT:utility.obj
 0003:000007d8       ?module_local_atexit_table@@3U_onexit_table_t@@A 000000018000c7d8     MSVCRT:utility.obj
 0003:000007f0       ?module_local_at_quick_exit_table@@3U_onexit_table_t@@A 000000018000c7f0     MSVCRT:utility.obj
 0005:00000060       $R000000                   000000018000e060     net.dll.res
